:1000000077C5000092C5000090C500000C941E3317
:100010008CC500008AC5000088C5000086C50000A8
:1000200084C5000082C500000C94F92F0C94E130C7
:100030000C941D1D7AC5000078C5000076C500002F
:1000400074C5000072C5000070C500006EC50000D8
:100050006CC500000C94D52F68C5000066C5000073
:1000600064C5000062C5000060C500005EC50000F8
:100070005CC500005AC5000058C5000056C5000008
:1000800054C5000052C5000050C500004EC5000018
:100090004CC500004AC5000048C5000046C5000028
:1000A00044C5000042C5000040C5000005010980AC
:1000B000A101850319012AB700150126B700950192
:1000C00075108100C0050C0901A101850419012AE0
:1000D000A002150126A002950175108100C005013E
:1000E0000906A1018506050719E029E71500250184
:1000F0009508750181020507190029EF15002501F2
:1001000095F075018102050819012905950575010C
:100110009102950175039101C00660FF0961A1017B
:100120000962150026FF00952075088102096315F4
:100130000026FF00952075089102C005010906A15F
:1001400001050719E029E7150025019508750181CA
:10015000029501750881010507190029FF15002680
:10016000FF0095067508810005081901290515008D
:100170002501950575019102950175039101C0094D
:10018000025B00030100A0FA090400000103010161
:100190000009211101000122440007058103080024
:1001A00001090401000203000000092111010001FE
:1001B0002222000705820320000107050303200017
:1001C00001090402000103000000092111010001DE
:1001D000226D0007058403200001120100020000C7
:1001E000000832FC87020100010200010C035300E9
:1001F0006F0066006C00650000001A034A006F0083
:100200007300650066004100640061006D006300DA
:1002100069006B0000000403090446001E001F0073
:10022000200021002200290014001A0008001500F7
:1002300017002B0004001600070009000A000057F1
:100240001D001B00060019000500E300E200E000AD
:10025000777C2800A8004C002700260025002400F9
:1002600023002A00130012000C0018001C002F00AD
:1002700033000F000E000D000B00E50038003700C2
:10028000360010001100E700E600E400787C2C0046
:10029000447E3A003B003C003D003E003F00010030
:1002A0001E021F02200221022202010014142D004E
:1002B0005700340032000100351435022D1455006A
:1002C00000000100010001000100010001004500E3
:1002D0004400430042004100400001002702260282
:1002E0002502240223020000320234026402640068
:1002F000350001002E02341430142D022E000100AE
:1003000001000100010001000100010000000000E7
:10031000000000000000010000000000520000008A
:100320004A0001000000500051004F004D00010044
:1003300000000000000000000000010001000100BA
:1003400001000100010001002202610060005F0065
:100350000000010055005E005D005C0000005700D9
:1003600024025B005A0059000000560027023700A3
:1003700036006200000001000100010001000100E0
:10038000010001000000000000000000000001006A
:100390000000000000000000427801004578477826
:1003A00049784B7843780100467848784A784C7809
:1003B0000000010001000100010001000100000037
:1003C000000000000000000000000000000000002D
:1003D000000000000000007C0000500900005009EF
:1003E000000000000000AB00AE00AC000000010007
:1003F00001000100010001000100A900AA004B005A
:100400004E00010001000100010001000100010097
:1004100001000100010001000100000000000000D7
:1004200000000000000000000000000000000000CC
:100430000000000000000000000000000000FC02BE
:100440000202028242428202C242424202C242424C
:100450004202020202FC0000000000000000FF0057
:100460000000000F10100F001F020200001F020208
:100470000000000000FF000000000000000001027A
:10048000020202020202020202020202020202024C
:100490000202020202010000000000000000007CD5
:1004A0008282824400F8242224F800FE1212120CE8
:1004B000004C9292926400000000000000000000D6
:1004C000000000000000000000000000000000002C
:1004D0000000000000000000000000000000FCFE22
:1004E000FEFEFE7E3E9E9E3E7EFE1E1EFEFE1E1EEC
:1004F000FEFEFEFEFEFC0000000000000000FFFF0C
:10050000FFFFFFF0E0CFCFE0F0FFC0C0FCF9C0C0BC
:10051000FFFFFFFFFFFF00000000000000000103DD
:10052000030303030303030303030303030303039B
:100530000303030303010000000000000000007C2F
:100540008282824400F8242224F800FE1212120C47
:10055000004C929292640000000000000000000035
:10056000000000000000000000000000000000008B
:1005700000000000000000000000000000000C0A65
:1005800009894929190981412111C93F0F01013107
:10059000190F8442211109050301C0A090888482AB
:1005A00081909894929190F0FC838080E01CFC8074
:1005B000808087F8000000000000808080808080BC
:1005C000808080808080808080808080808080802B
:1005D000808080808080808080800000000000001B
:1005E0000000FF01010101F19191916101010101FF
:1005F00001FF0000000000000000000000000000FB
:100600000000FF808080808F80818284888080804D
:1006100080FF00000000000000000000000000005B
:100620000000FF01010101F10101010101010101CE
:1006300001FF0000000000000000000000000000BA
:100640000000FF808080808F8888888880808080FC
:1006500080FF000000000000000000AE00AF0001BD
:100660000101010101010101020202020202020272
:100670000203030303030303030404040404040444
:100680000505050505060606060607070707070808
:10069000080808090909090A0A0A0B0B0B0C0C0CBB
:1006A0000D0D0D0E0E0E0F0F0F1010111111121255
:1006B00013131414151516161717181819191A1AD2
:1006C0001B1B1C1D1D1E1E1F202021222223242433
:1006D000252626272829292A2B2C2D2D2E2F30316F
:1006E0003232333435363738393A3B3C3D3E3F4081
:1006F0004142434445464748494A4C4D4E4F50516C
:100700005354555658595A5B5D5E5F616264656625
:1007100068696B6C6D6F7072737577787A7B7D7EAC
:100720008082838587888A8C8E8F91939596989AFC
:100730009C9EA0A2A3A5A7A9ABADAFB1B3B5B7BA14
:10074000BCBEC0C2C4C6C9CBCDCFD1D4D6D8DBDDE8
:10075000DFE2E4E7E9EBEEF0F3F5F8FAFDFF00DAAB
:100760000281FFD9F1DB20A4A62EAF00A0C0D300E8
:1007700000A1C8D30000AED580A81F408D14200072
:100780000000000000000000000000000000000069
:100790000000000000000000000000000000000059
:1007A000000000007E0F00D4FFFFFFC700000078AC
:1007B00000000000000000002A2B280000000000BC
:1007C0000000000000000000000000290000000000
:1007D0002C1E3420212224342627252E362D37386E
:1007E000271E1F202122232425263333362E373877
:1007F0001F0405060708090A0B0C0D0E0F10111235
:10080000131415161718191A1B1C1D2F3130232D00
:10081000350405060708090A0B0C0D0E0F101112FE
:10082000131415161718191A1B1C1D2F3130354CAF
:1008300081422408102040808040201008244281FA
:10084000814224100804020101020408102442819C
:1008500081C2E4F0F8FCFEFFFFFEFCF8F0E4C28188
:100860008143270F1F3F7FFFFF7F3F1F0F274381DC
:10087000010204081020408080402010080402017A
:100880000103070F1F3F7FFFFF7F3F1F0F0703017C
:10089000804020100804020101020408102040805A
:1008A00080C0E0F0F8FCFEFFFFFEFCF8F0E0C08046
:1008B00000000000000000005F00000000070007CB
:1008C0000000147F147F1400242A7F2A12002313AF
:1008D00008646200364956205000000807030000F3
:1008E000001C224100000041221C00002A1C7F1C29
:1008F0002A0008083E080800008070300000080840
:1009000008080800000060600000201008040200D1
:100910003E5149453E0000427F400000724949492E
:1009200046002141494D33001814127F100027451D
:10093000454539003C4A4949310041211109070028
:10094000364949493600464949291E00000014002D
:10095000000000403400000000081422410014147C
:100960001414140000412214080002015909060061
:100970003E415D594E007C1211127C007F4949496D
:1009800036003E41414122007F4141413E007F49C6
:10099000494941007F09090901003E414151730065
:1009A0007F0808087F0000417F4100002040413F50
:1009B00001007F08142241007F40404040007F0238
:1009C0001C027F007F0408107F003E4141413E0031
:1009D0007F09090906003E4151215E007F0919295E
:1009E000460026494949320003017F0103003F4088
:1009F00040403F001F2040201F003F4038403F0044
:100A00006314081463000304780403006159494D1A
:100A10004300007F414141000204081020000041D2
:100A200041417F0004020102040040404040400078
:100A30000003070800002054547840007F284444F5
:100A40003800384444442800384444287F0038544F
:100A50005454180000087E09020018A4A49C7800D1
:100A60007F080404780000447D4000002040403DA1
:100A700000007F102844000000417F4000007C04FB
:100A8000780478007C080404780038444444380032
:100A9000FC182424180018242418FC007C080404E2
:100AA000080048545454240004043F4424003C40AB
:100AB00040207C001C2040201C003C4030403C007A
:100AC0004428102844004C9090907C004464544C7E
:100AD000440000083641000000007700000000419B
:100AE000360800000201020402003C2623263C00D6
:100AF00011241FBECFEFDAE0DEBFCDBF13E0A0E0D0
:100B0000B1E0E0ECFAE602C005900D92AA38B10718
:100B1000D9F729E0AAE8B3E001C01D92A63AB207CE
:100B2000E1F70E94582A0C94F4346ACAEF92FF92BB
:100B30000F931F93CF93DF93D22F4934D8F5C42F4F
:100B4000C695C695C695477020E2C29FD001112474
:100B500070E06A59774FA60FB71F60E070E028E099
:100B600030E0241B3109FC01E60FF71FE4915D9191
:100B70000E2F10E0FD0131977F01E02F042E01C000
:100B8000EE0F0A94EAF75E2BF7015083411571F0DE
:100B9000C93061F0F801022E02C0F595E7950A947C
:100BA000E2F75F965C915E2B5C935F976F5F7F4F80
:100BB0006D17C8F2CDB7DEB7E6E00C9465349C0142
:100BC00091509F31B8F4832F817034FF0BC0829510
:100BD000807F31FD806232FD806433FD8068FB01DF
:100BE0000995089531FD826032FD846033FFF7CFAF
:100BF0008860F5CF80E0F3CF982F92959F7061F4D5
:100C000020E0982F892F8695869511F02E5F982FDA
:100C1000892F8695820F089524E0F4CF80930B08E6
:100C2000089580930C08089521E001C0220F8A9551
:100C3000EAF780910C08822BF4CF21E001C0220F4B
:100C40008A95EAF7822F809590910C088923E9CF45
:100C5000CF93C1E061FDC4E060FDCC0F62FDC295A1
:100C600093E0769567959A95E1F79B01220F331FE4
:100C7000260F371F420F531FFA0140E050E090E06B
:100C80006191DF019C01042E02C0369527950A94DC
:100C9000E2F72695220B26272C2326272E934F5F3B
:100CA0005F4F4330510561F7CF910895A82FA7708A
:100CB00023E0969587952A95E1F79C01220F331F33
:100CC000820F931F680F791FFB0140E050E080E026
:100CD000219130E00A2E02C0369527950A94E2F75A
:100CE0002170042E01C0220F0A94EAF7822B4F5F75
:100CF0005F4F4330510561F70895282F862F9A30B2
:100D000068F4263050F4622F70E026E0929F600D68
:100D1000711D11244AEE57E09BCF08959C5F9230DD
:100D2000E0F7622F70E047EE57E0F6CF292F9A30B8
:100D300058F4863080F490E06AEE77E036E0239F46
:100D4000800D911D1124B2CF2C5F223020F467EE6C
:100D500077E090E0F8CF80E0089590910C0821E0D2
:100D600030E0F90101C0EE0F8A95EAF7D90101C020
:100D7000AA0F6A95EAF7EA2B01C0220F4A95EAF713
:100D8000892F8E23E81303C0892F822B4ACF209509
:100D9000822F8923FBCFE091120890911108E9136B
:100DA00002C080E008959F0157E0E59FF001112403
:100DB000ED5EF74F5181561306C05081581303C0A2
:100DC0005581541305C02F5F3F4FF901E770E7CFFE
:100DD00081E008958091120820911108281301C024
:100DE000089501968770FACF90910D088095892318
:100DF00080930D08282F277061F4891751F0909186
:100E00000F0892FF06C086958695869516DF10928C
:100E10000D0808958091080890911008892B9091F1
:100E200009089115C9F0892B90918E01913021F418
:100E300090910E0897FD11C096E02EE833E040E057
:100E40009150F90150812F5F3F4F51114F5F911128
:100E5000F7CF41111092090808959EE126E933E089
:100E6000EECF8095982F80910808892380930808F9
:100E70000895803E9105D1F1C8F48133910509F4BC
:100E800081C048F48932910509F471C08A32910514
:100E900009F47FC0089589339105E1F08238910506
:100EA000C9F08533910509F45DC00895843E91052C
:100EB000D1F148F4823E910531F1833E910541F133
:100EC00081EE90E00895863E9105C1F1873E91053F
:100ED000F1F1089520910E08237009F064C020916B
:100EE0000F0823FF14C089E290E0089520910E08B6
:100EF00020FD45C030910F0830FF09C024FD24C0FB
:100F000083EE90E0089520910E0822FDF7CF08951A
:100F100020910E0822FD44C030910F0830FD43C0DF
:100F200024FFF5CF11C020910F0821FFF0CF809151
:100F30000E0884FD09C087EE90E0089520910E0808
:100F400023FFE5CF24FFF7CF80E090E008952091C4
:100F50000E0823FD2BC030910F0831FFE1CF84EE46
:100F600090E0089520910E0825FFD1CFBCCF2091AD
:100F70000E0825FD1EC020910F0823FFC8CF89E36E
:100F800090E0089520910E0826FFC1CF8AE290E0FC
:100F9000089520910E0826FFBACF81E390E00895CE
:100FA00082EE90E0089580EE90E0089586EE90E065
:100FB000089585E390E0089590910E0892FF10C087
:100FC00041E0282F2471243009F040E031E0282F3F
:100FD0002871283009F030E0431711F02CE0822707
:100FE00093FF10C041E0282F2471243109F040E024
:100FF00031E0282F2871283109F030E0431711F033
:101000002CE0822730910F0830FF10C051E0282FCC
:101010002171213009F050E041E0282F287128305B
:1010200009F040E0541711F029E0822731FF10C089
:1010300041E0282F2171213109F040E031E0282FD3
:101040002871283109F030E0431711F029E0822798
:1010500094FF02C083FD877E08950F931F93CF9363
:10106000DF9307DFEC01D23508F04DC0D03508F032
:10107000C3C0C03ED10530F5CD3CD10508F09AC0C3
:10108000C83AD10578F4C53AD10508F090C0C1300E
:10109000D10599F1CE010497813A910570F1C0E034
:1010A000D0E02BC0CE01885A91094B97C0F7C85A9F
:1010B000D0E0CC0FDD1FC25EDC4F0990D881C02D7F
:1010C000D4641BC0D03490F4D03208F0A8C0C83E1D
:1010D000D10598F0CE0191509F3108F78D2F6CDF2C
:1010E000082F8C2F90E0C5DE902B54C08C2F90E001
:1010F000C0DEDF70C82FD92BD06ACE01DF91CF912F
:101100001F910F910895C03882E5D807B8F5C03611
:1011100082E5D80708F056C0C03482E5D807C8F485
:10112000C03282E5D80708F047C08C2F8695869597
:1011300020E2829FC0011124C37021E030E002C090
:10114000220F331FCA95E2F7E901C82BD92BDD68BE
:10115000D4CF8C2F86958695877020E2829FC00120
:101160001124C37021E030E002C0220F331FCA9562
:10117000E2F7E901C82BD92BDC68BFCFC03C82E580
:10118000D80750F48C2F8F71C03AD24580F5982F34
:1011900084EF906AEC01B1CFCE01805C92458097DC
:1011A00008F07DCFDC2FDF71C0EFD06AA6CFA49707
:1011B000D064A3CFD065A1CF8C2F8F71D82FC1EF72
:1011C000D06A9BCF8C2F86958695877020E2829F70
:1011D000C0011124C37021E030E002C0220F331F90
:1011E000CA95E2F7E901C82BD92BDA6886CFE4DE8D
:1011F000C0E0D82FD06281CF8C2F8F71DDDE93E0DD
:10120000CC0FDD1F9A95E1F7DF70282F84FF04C013
:1012100090E1899F90011124C22FD0696ECF8D2F4C
:101220008F71CADE082F8C2F90E023DE902BEC010B
:10123000E1CF80E00895F894E82FE295EF70F0E0B8
:1012400041A18F7021E001C0220F8A95EAF7922F09
:101250009095942391A392A1822F892B82A37894B5
:10126000089581E0809333070895CF92DF92EF9243
:10127000FF921F93CF93DF93462F172FE82FF0E0B5
:10128000E25AF94F71110CC0E4918E2F7E2F6E2F10
:10129000DF91CF911F91FF90EF90DF90CF90089555
:1012A000F491EF2F86E0689FE00111242FEF30E0EA
:1012B000CE01B9010E942934DB01CA01880F991FB0
:1012C00065E56A9FA0016B9F500D1124841B482F78
:1012D000440F480FC901811B9109F89F7001F99FC4
:1012E000F00C11248F2D149FB0011124672F70E092
:1012F0006901C61AD70AB601F69F6001F79FD00CA4
:101300001124A330B10549F1B901641B7109AB0186
:10131000149FB001159F700D1124672F70E0261BDC
:10132000370BF29FA001F39F500D1124752FCC3F76
:10133000D34050F4A130B105A1F0129709F0A7CF26
:10134000EF2D852F7F2FA3CFA430B10569F016971D
:1013500009F49DCF7F2D8D2D9ACF7D2DEF2D8F2FD1
:1013600096CF7F2FED2D93CFE52F7F2DF8CF982FA0
:101370008091B607811529F081E0943208F080E071
:10138000089581E09834FACF9C0180E090E0269F98
:10139000020E811D369F800D911D1124830F911D1A
:1013A0000895409113015091140125E038E0429FC7
:1013B000C001439F900D529F900D1124875E994C60
:1013C0008093130190931401890F0895982FE82FAB
:1013D00096FDE0958E2F8F7096FD8F5FE695E695D2
:1013E000E695E670F0E0E353FD4F2181289F202D24
:1013F000812D112422952F708295807F282B80814A
:10140000820F97FD8195805808951F93CF93DF93A6
:10141000EB01182F822F8695D9DF805887FD8195A3
:10142000880F282F219F020E20E0211D1124822FDA
:10143000BE01DF91CF911F910895622F0895E42F8F
:10144000F0E0EE0FFF1FEB50FE4F6081621B08952E
:101450000F931F93022F50E0FA01EE0FFF1FE75486
:10146000FE4FE5ADE052E7FDE195440F551F4B50AF
:101470005E4FDA012C91201B310B2E0F620F1F9152
:101480000F9108950F931F93A02FB0E0FD01EE0F71
:10149000FF1FE754FE4F05AD0052110B2003F00172
:1014A000219FF00D1124AA0FBB1FAB50BE4F2C91F2
:1014B0002057330B4203D001439FB00D11249F01ED
:1014C0002A0F3B1F12F421583F4F220F232F221FB8
:1014D000330B620F1F910F9108959091E904982B9F
:1014E0009093E90408953091B607311521F08432C4
:1014F00091052CF008958432910514F08497E2C38D
:1015000008951F93CF93DF93C82FD0E0FE01EB57D0
:10151000FD4F808190911101892389F042DF182FBE
:1015200040DF20E8829FC0011124792F7158612F7C
:10153000809187079ADE472F282FCE01D4DFDF91D5
:10154000CF911F910895FF920F931F93CF93DF9335
:10155000182F062FF42EC0E0D0E02F2D402F612F42
:10156000CE01C1DF2196C834D105B9F7CDB7DEB7BA
:10157000E5E00C946634982F990F990F890F982FF6
:101580009B5F993408F098E42091B607211104C0BC
:10159000843228F484E20895953208F094E20895A4
:1015A000EF92FF920F931F93CF93DF937C01809173
:1015B0001001E1DFC82F192F6091880766956695A5
:1015C00021E0620F08F46FEF8091E5049091E6044A
:1015D000DBDE082FD0E0812FC11730F0C8DECDB799
:1015E000DEB7E6E00C946534FE01EB57FD4F8081D9
:1015F00090911101892379F0609185077091860798
:1016000080918707202F4C2FF70109952EDE472F59
:10161000282FCE0168DF2196DECFA0E0B0E0E3E125
:10162000FBE00C944734182F80910F01811324C0E4
:1016300090918407937020910E0130E081E0921721
:10164000130609F480E0809312018091890790913C
:101650001101981731F08093110140E060E080E0C3
:1016600072DF193058F4E12FE150E830E8F4F0E08F
:10167000EA50FB4C0C94873481E0E5CF1F3F09F41E
:101680003EC180E0909110019F5F90931001811105
:101690005FC182E080930D0180911201811158C1D8
:1016A000111156C183E052C180911201811549F395
:1016B00040E060E080E047DFE4CF809110015BDF35
:1016C000C82F092F60918507709186078091870741
:1016D000CCDDF62EE72ED82ED0E00C1709F018F44A
:1016E000802F45DECFCFFE01EB57FD4F80819091DB
:1016F0001101892329F02D2D4E2D6F2DCE01F3DE02
:101700002196EBCF85E09AE04BDFBCCF8DE19AE0EC
:10171000FBCF8FE19AE0F8CF88E29AE0F5CF809195
:10172000100129DFC82F092F6091880766958091E5
:10173000E5049091E60428DED82ED0E0CE01880F93
:10174000991F87549E4F7C010C1751F248F2FE01FD
:10175000EB57FD4F808190911101892309F44FC00F
:10176000F70144AD4057550B85AD8052990B449F0E
:101770009001459F300D300D1124889FA001899F55
:10178000500D500D1124240F351F822F22303105AA
:1017900020F19FEF213E8EE1380740F4C901E5E0DA
:1017A00096958795EA95E1F7982F985F61E0462F27
:1017B000490F5527551F55954795842F449FF00194
:1017C000459FF00DF00D11242E173F07E8F4942FDC
:1017D0009150961760F7862F815090E0BC01660FFC
:1017E000771F680F791F759567956D0D7091860746
:1017F000809187073ADD472F282FCE0174DE21968E
:1018000082E0E80EF11CA0CF4F3F39F3642F6F5FE9
:10181000E0CF80911001AFDEC82FF92E60918807CC
:10182000669566958091E5049091E604ADDDE82E1D
:10183000805CCCDD8058D82E8E2DC8DD8058C82E17
:10184000D0E0CF1510F08F2D4CCFFE01EB57FD4FA0
:10185000808190911101892379F0609185077091C1
:101860008607809187070C2F2C2D4D2D0BDEFDDC7C
:10187000472F282FCE0137DE2196E3CFC0911001EC
:10188000C1111DC06091880720E1620F08F46FEF5D
:101890008091E5049091E60477DD65E070E00E94B8
:1018A0002934892B61F47DDD28E4829FA001112475
:1018B000852F880F880B50930B0180930C018C2F80
:1018C0005ADEEC0190911201911115C020910B018B
:1018D00030910C012817310580F02D17310568F47F
:1018E000822F0FDE89E480930B0110920C0105C05A
:1018F0008C2F07DECF5FCD17D8F38D2FF2CE9091CE
:10190000E604A091E704B091E804892F9A2FAB2F49
:10191000A69597958795A69597958795837090E05E
:10192000A0E0B0E082309105A105B105B1F08330AF
:101930009105A105B105A1F040E060E0109790404D
:10194000814081F464E180E0FEDD82E080930D015E
:10195000CDB7DEB7E8E00C94633444E160E0F3CF48
:1019600044E164E184E1F0CFCF93C82F811581F089
:1019700080911E0781110CC050DE10920F018091E2
:101980008407837080930E0163D583E080930D01FB
:10199000C0931E07CF9108959091840721E092276C
:1019A0009093840710920D0198CD809184078370E5
:1019B00011F410920D01809184078C7F81608093D7
:1019C0008407089580918407837011F010920D01AF
:1019D000809184078C7F8093840708959091840779
:1019E000937091F0811589F0893088F48F73880F96
:1019F000880F982F209184072370922B909384074F
:101A000010920D01862F69CD089581E0F0CF88E016
:101A1000EECF80918407869586958F5F893008F098
:101A200081E061E0DBCF80918407869586958150C7
:101A300009F488E061E0D2CF90918407937059F067
:101A40008093850760938607493708F048E74093FD
:101A50008707822F42CD0895E4E8F7E0818190E086
:101A600021E0438162810896E7CFE4E8F7E08181D5
:101A700021E0438162818850990BDECFE4E8F7E0F2
:101A8000628120E1620F08F46FEF818121E04381E0
:101A900090E0D2CFE4E8F7E0628120E1621B08F435
:101AA00060E0818121E0438190E0C6CFE4E8F7E087
:101AB000438120E1420F08F44FEF818121E06281F0
:101AC00090E0BACFE4E8F7E0438120E1421B08F45C
:101AD00040E0818121E0628190E0AECF20918807D3
:101AE00030E1230F08F42FEF2093880781E0F5CC35
:101AF0002091880730E1231B08F420E02093880719
:101B000081E0EBCCE0918907EF3F69F0E53069F0C7
:101B1000E23069F4EF5FF0E0EB54FE4F8081809398
:101B2000890781E0DACCE0E0F5CFE1E0F3CFE0E057
:101B3000F2CFE0918907EF3F91F0E53071F0E230AC
:101B400019F0E1110EC0E3E0E150F0E0EB54FE4F7C
:101B500080818093890781E0C0CCE1E0F5CFE3E0AC
:101B6000F4CFE0E0F2CF2091F406382F3203C00129
:101B70001124923014F080E090E082519B4F8093CA
:101B8000EC049093ED0408950F931F93CF93DF938C
:101B9000A091EC04B091ED049D012E5E3440620FE3
:101BA000731F613042E0740710F060E072E0409112
:101BB000EA045091EB04FC0101E010E0261737071E
:101BC00048F04093EA045093EB04DF91CF911F91CA
:101BD0000F91089584919D91981789F0ED018A9352
:101BE000C901C5E096958795CA95E1F7E80102C05D
:101BF000CC0FDD1F8A95E2F7CE014C2B592B2F5FBE
:101C00003F4F3196DBCF90917907292F30E07091CB
:101C10007A07A9014395437050E07417150689F0BF
:101C20002958384F60FB87F9F90184839F5F9370CF
:101C300090937907809177078F5F8093770781E092
:101C4000089580E0089590E06115D1F08A5E9E4F7E
:101C5000FC0180818F3F99F0E82FE295EF70F0E072
:101C600041A18F7021E001C0220F8A95EAF7922FDF
:101C70009095942391A392A1822F892B82A30895FA
:101C8000895E9E4FE5CF90E06115A9F08A5E9E4F78
:101C9000FC0120812F3F91F0E22FE295EF70E05E92
:101CA000F0E0808190E02F7002C0959587952A958D
:101CB000E2F781700895895E9E4FEACF80E0089533
:101CC000539A0895FC01EE0FFF1FE80FF91FEA5128
:101CD000FC4F6183408322830895FC01680F791FC4
:101CE0008FEF41E39191892728E030E0982F990FF9
:101CF00087FF09C0892F842721503040B9F7E617A4
:101D0000F70781F70895892FF7CF811144C0EFECD1
:101D1000F3E020E030E047E0429FC001439F900D98
:101D20001124DC01AC52BC4F5C9153FF06C05681BC
:101D3000511103C081539C4F08952F5F3F4F379639
:101D40002330310549F7611531F18091D40383FFC8
:101D50001CC08091DB0383FF1BC08091E20383FDE5
:101D60001AC082E090E027E0289FF001299FF00D43
:101D70001124CF0181539C4FDC0116961C92EC522A
:101D8000FC4F208128602083089580E090E0EBCF15
:101D900081E090E0E8CF80E090E0089541155105A2
:101DA00011F0FA01099508958091B507811103C0DA
:101DB000809183070895E091DD07F091DE07309769
:101DC00039F00190F081E02D309711F009950895D8
:101DD00080E00895A3E0B0E0E0EFFEE00C944D3425
:101DE0002091CD033091CE0328173907B1F08093AD
:101DF000CD039093CE03E091DD07F091DE0730979D
:101E000061F00084F185E02D309739F023E02983DB
:101E10008A839B83CE01019609952396E2E00C9478
:101E20006934A3E0B0E0E7E1FFE00C944D34209189
:101E3000CB033091CC0328173907B1F08093CB0343
:101E40009093CC03E091DD07F091DE07309761F0CD
:101E50000084F185E02D309739F024E029838A83CE
:101E60009B83CE01019609952396E2E00C94693498
:101E700090918E01913099F0AEE8B3E0EFEF90E0F1
:101E80002C91821759F01196EF3F19F4211101C0DE
:101E9000E92F9F5F9630A1F7EF3FC1F4089590912D
:101EA0000E0897FFE9CFE82FE695E695E695803F87
:101EB000A8F7F0E0EC56FC4F877021E001C0220F3C
:101EC0008A95EAF78281822B82830895FE2FFF0F85
:101ED000FF0BE457FC4FF8CF90918E01913021F425
:101EE00090910E0897FD0CC0EEE8F3E091918913F4
:101EF00002C0DF011E9293E0E439F907B9F70895B3
:101F0000E82FE695E695E695803FC8F7F0E0EC56B9
:101F1000FC4F9DEF81FD97EF80FF959582FD929597
:101F2000828189238283089580918D0108952FB73E
:101F3000F8946091C7037091C8038091C903909190
:101F4000CA032FBF08958091B507811539F0EFDFDF
:101F5000462F572FBC01CB01BA010895E8DFDC0101
:101F6000CB014091B7075091B8076091B9077091C4
:101F7000BA07480F591F6A1F7B1FEDCF87E797E706
:101F8000809300089093010888E19AE00FB6F894D6
:101F9000A895809360000FBE90936000FFCF0895D6
:101FA000FC012091BD033091BE032617370748F08E
:101FB0006115710529F49091E8009E779093E800EF
:101FC0009B0190E02115310541F4911106C08091EB
:101FD000E80082FF32C080E00895809114078115E7
:101FE000C1F18530C1F18091E80083FD30C080915E
:101FF000E80082FDECCF8091E80080FFE3CF809184
:10200000F3004091F200582F2115310519F04830A6
:10201000510558F091E04830510509F090E04091A9
:10202000E8004E774093E800CDCF81918093F10096
:10203000215031094F5F5F4FE7CF80911407811521
:1020400041F0853041F08091E80083FFC0CF81E00E
:10205000089582E0089583E00895982F9093E90011
:10206000891771F07091EC002091ED005091F00013
:1020700021FD09C09F5F973089F78093E90008959B
:10208000762F242F50E03091EB003E7F3093EB0011
:102090003091ED003D7F3093ED003091EB003160E9
:1020A0003093EB007093EC002093ED005093F00020
:1020B0002091EE0027FDDECF08958091B70387FFC2
:1020C00013C08091E80082FF06C08091E8008B7702
:1020D0008093E8000895809114078111F2CF08954C
:1020E000809114078115D9F38091E80080FFF8CF23
:1020F0008091E8008E77ECCF2091E4003091E500EC
:1021000095E6A9012091EC00822F817020FF06C086
:102110008091E80080FF06C080E008952091E800EB
:1021200022FD1AC080911407811589F0853089F04D
:102130008091EB0085FD0FC02091E4003091E50017
:1021400042175307F9F29150E1F684E0089582E0D6
:10215000089583E0089581E00895CF93DF93C8ED5B
:10216000D0E088818F7E8883E7EDF0E08081816018
:10217000808384E082BF81E08093B60388818E7F74
:102180008883E2EE10821092DA00A1EEB0E01C9299
:1021900088818F77888388818068888388818F7D14
:1021A000888319BC109214071092B5031092F70699
:1021B0001092B403A0EE8C918B7F8C938881816008
:1021C000888342E060E080E048DFA1EEB0E08C91DF
:1021D0008E7F8C93E2EEF0E080818160808380814D
:1021E00088608083E0EE80818E7F8083888180613B
:1021F0008883DF91CF910895E8EDF0E080818E7FB4
:1022000080831092E2001092DA001092E100A0EEBA
:10221000B0E08C9181608C9380818F77808319BC32
:10222000A7ED8C918E7F8C9380818F7E808310921E
:10223000B6030895A0E0B0E0E0E2F1E10C9443348D
:10224000D82E80919A018D1549F000916408109163
:1022500065080115110539F4D0929A01CDB7DEB7A2
:10226000ECE00C945F348D2D0E94FC05B82E90910B
:10227000630880E0891781F3F8012081B21609F420
:1022800055C08F5F0B5F1F4FF5CFF8010180F281C2
:10229000E02DEE0DFF1D2081822F81568A31B8F48A
:1022A00020522052330B46E0429FC001439F900DC5
:1022B000112425E0492D62E08055974F0E94960534
:1022C0008FEFE81AF80A892D865F982E65C02032B4
:1022D00040F720E2E6CFED120FC0A814B90401F5D3
:1022E00080E898E020E14C2F60E10E9496058FEF96
:1022F000E81AF80AC85F6CC0C7010197A816B906AA
:1023000091F080E598E0AE14BF0461F31F3F29F01F
:1023100080E398E0AE14BF042CF380E498E0E2CFB1
:1023200080E798E0DFCF80E698E0DCCF8181928182
:10233000892B09F491CFD0916208D11509F48CCF83
:10234000E6E6F8E080E491E011920197E9F7F80100
:10235000A181B281FD0101900020E9F73197EA1BCC
:10236000AE2ECD2EC3944AE04E9F402D11244250F4
:1023700080E590E09C01241B3109A9015595479502
:10238000942E2C2D220F220F220F821B910995953E
:102390008795C82FE12CF12CEA1408F476CFE2E5FA
:1023A000F8E010E0A081B181109719F08C918B15A5
:1023B00029F032961F5F1D13F5CF1FEFE12CF12C92
:1023C000A12EB12EBB0CBB088D2F8150990B4C0157
:1023D000EC1408F041CFE1107ECF80EA98E01115AF
:1023E00009F480CF80E998E07DCFA0E0B0E0EBEF8A
:1023F000F1E10C9445347C016B015A0180919807FE
:102400000AE010E08A3010F001E010E0C1E0D0E016
:10241000B601C701F5010995811115C021960C1768
:102420001D078CF0CC9F9001CD9F300D300D1124F5
:1024300080E090E045E34A95F1F7000001968217AD
:102440009307C1F7E5CFCDB7DEB7EAE00C9461346E
:102450003BB1377F2BB128604FB7F89486EE93E0FD
:10246000FC010196508168E02BB9000000C057FFC5
:102470003BB9550F000000C000C000C03BB900C010
:102480006A9591F754E08E3B950751F74FBF8FE562
:1024900094E00197F1F700C0000008950F931F9397
:1024A000CF93DF93EB018A0190911407943059F593
:1024B0008093E9008FEF9091E80095FD06C095EDBF
:1024C0009A95F1F700008150B1F78091E80085FFFF
:1024D0001AC012DE811112C08091E80085FD06C08D
:1024E0008091E8008E778093E800F3CF8881809315
:1024F000F1000150104011F02196EECF8091E800DC
:102500008E778093E800DF91CF911F910F9108950E
:10251000603229F440E250E0BC0182E0BFCF089570
:10252000CF93DF93EC0148E050E0BC0181E0B6DFDF
:1025300088E0FE01AFEBB3E001900D928A95E1F7E0
:10254000DF91CF91089540E250E0BC0184E0A6CF36
:1025500043E050E0BC0184E0A1CF90910F0892FBD2
:10256000222720F9281779F080FB92F990930F0821
:1025700060910E0870910F0884E090E00E94F034A2
:1025800082E00C94F40608951F93CF93DF93122FEB
:102590008630E0F46A30D0F44630C0F4C42FD0E086
:1025A000CC0FDD1F2CE0629FC00DD11D112498E7D8
:1025B000899FC00DD11D1124632FCE0189960E94E1
:1025C000D634612FCE018A960E94D634DF91CF9106
:1025D0001F9108950F931F93CF93DF93142F022F12
:1025E000863020F5623010F598E0899FE0011124D3
:1025F00024E0629FB0011124C60FD71FC750DD4FE2
:1026000081E08427632F9E01280F311D280F311D83
:10261000C9010E94D63481E090E0111102C083E02C
:1026200090E0602F8C0F9D1F0E94D634DF91CF91D8
:102630001F910F9108958F929F92BF92CF92DF9238
:10264000EF92FF920F931F93CF93DF939AEFC92ED0
:1026500093E0D92EE12CF12CC0E04701D0E018C066
:1026600021E030E0C43020F4F801859195919C017F
:102670004B2D6D2F8C2F88DFB3940E5F1F4F8B2D4A
:10268000863071F7DF5F86E0880E911CDA3039F012
:102690008401000F111F065E1D4FB12CE1CF860192
:1026A000D0E021E030E0C43020F4F801859195912C
:1026B0009C0141E06D2F8C2F8DDF21E030E0C43094
:1026C00028F4F8013296859195919C0140E06D2F98
:1026D0008C2F80DF8D2F0C5F1F4FD1E0813009F7E9
:1026E000CF5F88E0C80ED11C8CE3E80EF11CC63029
:1026F00009F0B3CFDF91CF911F910F91FF90EF9031
:10270000DF90CF90BF909F908F90089580918E0121
:10271000813069F580910E0887FF29C00E940A0761
:102720008093950340E250E06DEB77E084E993E01D
:102730000E949434892BD1F080E2E4E9F3E0ADEB20
:10274000B7E001900D928A95E1F7E091DD07F091F5
:10275000DE07309759F00480F581E02D309731F095
:1027600086E08093940384E993E0099508950E949C
:102770000A0780938C0348E050E06FED77E08CE827
:1027800093E00E949434892B89F388E0ECE8F3E02D
:10279000AFEDB7E001900D928A95E1F7E091DD078A
:1027A000F091DE07309711F30280F381E02D30972E
:1027B000E9F28CE893E0D9CF811531F090910808C7
:1027C000982B90930808A2CF0895811531F090912D
:1027D0001008982B9093100899CF0895811519F03F
:1027E0000E94310793CF0895811539F0809590911B
:1027F000100889238093100889CF0895CF93C82F9C
:102800008115C1F08450813A70F580918E0181303C
:1028100021F480910E0887FD0FC0EEE8F3E080817F
:10282000C817E9F0319683E0E439F807C1F78C2F37
:102830001FDB6CDFCF910895EC2FE695E695E695CA
:10284000F0E0EC56FC4F828190E04C2F477021E085
:1028500001C0220F4A95EAF78223892B41F38C2F7E
:102860003BDB54DFE4CF8C2F805E883060F4C77090
:1028700081E001C0880FCA95EAF7C0910808C82B0B
:10288000C0930808D6CF8C2F855A833028F48C2F1C
:102890008452990B9FDACECFC85ACB3158F6EC2F21
:1028A000F0E0EE0FFF1FEC5AFC4F80819181B9DA06
:1028B000C1CFCF93DF93EC01805E9109089720F0A0
:1028C00065EE73E1209711F46CED73E1CE010E9487
:1028D000DF058C2F93DFDF91CF910895CF93DF93A6
:1028E000EC018A81823039F4FB0182819381E1DF3E
:1028F0008D8182608D83DF91CF910895FB0180816E
:102900009181D7CF811511F1982F9450913A10F4FD
:10291000E3DAFCCE982F905E983058F4982F81E03F
:1029200091FD84E090FD880F92FD82950E94310711
:10293000F0CF982F955A933018F480E090E04ACA6F
:10294000885A8B3118F480E090E06BCA0895CF93D9
:10295000DF93EC01D7DFCE01805E9109089720F06C
:1029600064EF73E1209711F46EEE73E1CE010E94E3
:10297000DF05DF91CF910895FC018281813059F408
:102980008FE39CE90197F1F700C00000FB01808113
:102990009181DDCF08958230E9F7FB018281938137
:1029A000F8CF1F93CF93DF93182FEB0127DF8FE929
:1029B0009FE00197F1F700C000002197C1F7812F38
:1029C000A1DFDF91CF911F910895109208088091A7
:1029D0008E01813099F480910E0887FF0FC0E6E9DF
:1029E000F3E08EE111928A95E9F780E090E0F2D968
:1029F00080E090E016DA1092100888CEEEE8F3E05E
:102A000086E0F0CFE2DF88E19AE00FB6F894A8956F
:102A1000809360000FBE90936000FFCFAAE2B0E009
:102A2000E4E1F5E10C944C3487EB93E0FC01019672
:102A30002091F100208323E08F3B9207B9F780912A
:102A4000B803893009F457C0C8F4823009F4B3C020
:102A5000833009F483C0813081F18091E80083FFE5
:102A6000E7C08091B7039091B8039A3008F0E0C0B6
:102A7000E92FF0E0E250FB4C0C9487348A3009F4E3
:102A80008AC08B3051F78091B703813231F7809142
:102A9000BB039091BC03892B01F78091E800877FED
:102AA0008093E8000ADB81E09091B903911101C0A5
:102AB00080E080938E0189DFD0CF8091B703813A87
:102AC00061F68091E800877F8093E8008091BB03E6
:102AD0009091BC03892B59F060E080E090E070E0B9
:102AE0005FDA8091E8008B778093E800B6CF68E0EA
:102AF0008FEB93E0F4CF8091B703813209F0ADCF33
:102B00008091BB039091BC038D7F892B09F0A5CFE9
:102B10008091E800877F8093E8008091E80082FF41
:102B200018C02091F3008091F200922F029731F4A7
:102B30008091F100813011F0863021F48091F10014
:102B400080938D018091E8008B778093E800B5DA5F
:102B500084CF809114078111E0CF7FCF8091B7039C
:102B6000813A09F07ACF8091BB039091BC03892B05
:102B700009F073CF8091E800877F8093E80080910F
:102B8000E80080FFFCCF80918E018093F10080915E
:102B9000E8008E77DACF8091B703813209F05DCFFC
:102BA0008091E800877F8093E80087DA8091BA03FC
:102BB00080938C0152CF8091B703813A09F04DCFB9
:102BC0008091E800877F8093E8008091E80080FF93
:102BD000FCCF80918C01D9CF803889F0823841F5C3
:102BE0008091BB038F70873018F58093E900809146
:102BF000EB0085FB882780F91092E90006C08091E0
:102C0000F706880F9091B403892B9091E800977F85
:102C10009093E8008093F1001092F1008091E80019
:102C20008E7723C0811116C08091B903813009F1DC
:102C30008091E80083FF0AC08091E800877F80933D
:102C4000E8008091EB0080628093EB00AA96E3E0BD
:102C50000C946834823061F78091B903811579F062
:102C60001092E9008091E800877F8093E80025DAE0
:102C7000DFCF933009F080E08093F706F1CF8091A9
:102C8000BB038F70282F2150263090F68093E900E7
:102C90002091EB0020FFE4CF933031F48091EB00E2
:102CA00080628093EB00DCCF9091EB009061909379
:102CB000EB0021E001C0220F8A95EAF72093EA0099
:102CC0001092EA008091EB008860EBCF8111B0CFC9
:102CD0008091B9038F77182F8091E3008078812B42
:102CE0008093E3008091E800877F8093E800E5D936
:102CF0008091E80080FFFCCF8091E30080688093A2
:102D0000E30083E0111101C082E08093140790CFAB
:102D10008058823008F08CCF8091B9039091BA032B
:102D20008C3D23E0920789F583E08A838AE28983D8
:102D30004FB7F894DE01139620E03EE051E2E32F16
:102D4000F0E050935700849120FF03C082958F706C
:102D50003F5F8F708A30B8F0895C8D931D922F5F32
:102D6000243169F74FBF8091E800877F8093E800A6
:102D70006AE270E0CE01019613D98091E8008B776A
:102D80008093E80055CF805DE8CF292F30E02330D5
:102D9000310509F44DC078F52130310509F47CC0C6
:102DA0008BE590E0EFE7F1E02230310509F040CF0C
:102DB0002091E800277F2093E8002091BD03309107
:102DC000BE038217930708F49C0140E021153105EA
:102DD00009F067C0411165C08091E80082FDCDCF48
:102DE00080911407811549F2853039F28091E8000D
:102DF00083FFF2CFC2CF8091BB039091BC032132FD
:102E00003105D9F12232310509F012CF8330910515
:102E100008F00ECFFC01EE0FFF1FEF55FE4F0190A3
:102E2000F081E02D82569E4FDC018C9190E011C024
:102E3000282F30E0813089F022303105B1F0232B8A
:102E400009F0F6CEE6E1F2E0E4918E2F90E0E6E1C3
:102E5000F2E0009709F4ECCEABCFEAEFF1E0E491B9
:102E60008E2F90E0EAEFF1E0F4CFECEEF1E0E491A8
:102E70008E2F90E0ECEEF1E0ECCF8330910508F07E
:102E8000D7CE880F991FFC01E955FE4F0190F081C4
:102E9000E02D89E090E08CCF82E190E0EAEDF1E076
:102EA00087CF80911407811509F467CF853009F425
:102EB00064CF8091E80083FD60CF8091E80082FDBF
:102EC0008BCF8091E80080FF81CF4091F30080910B
:102ED000F200942F2115310519F08830910550F03A
:102EE00041E0089709F040E08091E8008E778093F8
:102EF000E8006CCF44914093F100319621503109A4
:102F00000196E8CF803809F093CE8091E800877F62
:102F10008093E8008091B5038093F1007FCE81110A
:102F200087CE8091B903182F823008F081CE80912E
:102F3000E800877F8093E8001093B503BED8111591
:102F4000D9F084E08093140742E061EC81E085D8F9
:102F500042E261EC84E081D842E261EC82E07DD81B
:102F600042E260EC83E079D880911407843051F418
:102F700082E080938F015CCE8091E30087FDE1CFFA
:102F800081E0E0CF81E0F5CFCF93DF93EB01FC014F
:102F90004481558160857185CE010E94CE0E9B8152
:102FA0009095809110088923809310088C810E944D
:102FB0003107ACDB87E019928A95E9F7DF91CF9171
:102FC00008950F931F93CF93DF938C01EB018D81B5
:102FD00081FD17C082608D83809110089B81892BB1
:102FE00080931008809108089C81892B80930808A1
:102FF0008DDBF8014281538160857185CE010E948D
:10300000CE0E10920208109203088D8180FD03C03D
:10301000BE01C801B9DFDF91CF911F910F910895D3
:10302000CF92DF92FF920F931F93CF93DF936901AB
:10303000E801082F880F110B41155105B1F0F80177
:1030400033E0EE0FFF1F3A95E1F7EC5DFE4F818113
:1030500092818A5B984FE0812E2F30E04E17510508
:1030600008F49A01A9010E94A134C8010E94BB334F
:10307000F82E8115E1F02097D1F0C80123E0880FE8
:10308000991F2A95E1F7FC01EC5DFE4F2381422F49
:1030900050E0C217D10508F4AE018C5D9E4FFC01D3
:1030A000648175816A5B784FC6010E94A1348F2DBF
:1030B000DF91CF911F910F91FF90DF90CF900895F6
:1030C000A4E0B0E0E6E6F8E10C944934E0902F0784
:1030D000F090300700913107109132070E94970F4E
:1030E000DC01CB018E199F09A00BB10B11E08436D6
:1030F0009105A105B10510F10E94A30FDC01CB01E0
:103100000296A11DB11D89839A83AB83BC8300E025
:1031100010E0980144E050E0BE016F5F7F4F86E011
:103120007FDF182F811551F00E94970F60932F07B2
:10313000709330078093310790933207812F249644
:10314000E6E00C946534A1E0B0E0E9EAF8E10C9423
:103150003D34662E2A01190168018D019E012F5F01
:103160003F4F40E050E0BA015BDF182F8115B1F10D
:10317000F20180809180A280B3800E94970F7980B5
:10318000681979098A099B096436710581059105D9
:1031900030F4B701C6010E946D0E8715F9F0870162
:1031A000910140E050E0BA01862D3ADF082FB701C7
:1031B000C6010E946D0E10E087110BC0102F117018
:1031C00000FF07C00E94970FF20160837183828322
:1031D0009383812F2196E2E10C945934A701B60123
:1031E000C1010E94A134F5CFA5E0B0E0EAEFF8E11B
:1031F0000C9447346B017D0107E417E0CE01019682
:103200009C0142E457E061E080E09DDF811559F0C8
:1032100095E09E012F5F3F4FF901ADE3B7E00190CC
:103220000D929A95E1F795E0EDE3F7E0D601019074
:103230000D929A95E1F72596E8E00C946334A8E0A6
:10324000B0E0E5E2F9E10C9449347D0102E517E0D4
:103250009E012F5F3F4F45E357E064E083E073DF5B
:10326000182F811599F19091510780913407981783
:1032700069F19091550780915407891709F1E92F59
:10328000F0E0E65BF84F848587FB662760F99F5F77
:10329000937090935507909153079F5F90935307B6
:1032A0008F770E94030EF82E8111E3CF00E010E02B
:1032B0009801A801B80185E0B3DEF8221F2D02C0F5
:1032C000F110F4CF8091510780933407812F289615
:1032D000E6E00C946534A0E0B0E0E1E7F9E10C949D
:1032E0004334D82EEB01C42E59014801E880F980FF
:1032F0000A811B810E94970FDC01CB018E199F0967
:10330000A00BB10B84369105A105B10510F4C114D1
:1033100079F000E010E09801A401B5018D2D80DE68
:10332000811539F00E94970F688379838A839B8384
:1033300081E0CDB7DEB7ECE00C945F340F931F93C0
:1033400041E090915E0780910C08981301C040E025
:1033500001E010E02CE038E06BE277E087E0BBDFD3
:10336000811571F041E090915F0780910B089813EF
:1033700001C040E02BE038E067E277E088E0ABDFB7
:103380001F910F910895A1E0B0E0E9ECF9E10C94F0
:103390004B3480911907898320916A0790E041E0BE
:1033A0002817190609F440E08D019E012F5F3F4F59
:1033B0006AE177E08BE08FDF2196E4E00C946734DC
:1033C000CF92DF92FF920F931F93CF93DF93F82E4C
:1033D0006B01EA01A801B901CE010E94943441E0D9
:1033E000892B09F440E09E01B6018F2D74DFDF9137
:1033F000CF911F910F91FF90DF90CF9008950F9381
:103400001F9305E010E02CE437E0AC0169E377E0BE
:1034100082E0D6DF1F910F910895A1E0B0E0E3E1D3
:10342000FAE10C944B340E94D40E898301E010E041
:1034300020E637E0AE014F5F5F4F63E277E089E05F
:10344000BFDF2196E4E00C946734A9E0B0E0EBE242
:10345000FAE10C944B3488E0E4E8F7E09E012F5F3A
:103460003F4FD90101900D928A95E1F780911E0797
:10347000898709E010E021E637E0CE010196AC0132
:103480006FE177E08AE09CDF2996E4E00C946734F2
:10349000ACE0B0E0EEE4FAE10C944B348091940798
:1034A00090919507A0919607B091970789839A8389
:1034B000AB83BC838091900790919107A091920774
:1034C000B09193078D839E83AF83B88780918C07DB
:1034D00090918D07A0918E07B0918F0789879A8769
:1034E000AB87BC870CE010E02BE637E0AE014F5F06
:1034F0005F4F65E177E08CE063DF2C96E4E00C94AD
:1035000067340F931F93CF93DF93863008F56A30AB
:10351000F8F44630E8F4C42FD0E0CC0FDD1F9CE077
:10352000699FC00DD11D112498E7899FC00DD11D41
:103530001124CE0189960E94BA34082FCE018A96B2
:103540000E94BA34902FDF91CF911F910F9108956F
:1035500080E090E0F8CFFF920F931F93CF93DF931B
:10356000F42E863048F5623038F598E0899FE00106
:10357000112484E0689FB0011124C60FD71FC750E3
:10358000DD4F81E084279E01280F311D280F311D5A
:10359000C9010E94BA34082F81E090E0F11002C006
:1035A00083E090E08C0F9D1F0E94BA34902FCDB71E
:1035B000DEB7E5E00C94663480E090E0F8CF7A3036
:1035C00038F4663060F4863050F4462F672F99CF78
:1035D0007D3F41F4623018F441E0863050F080E0E5
:1035E00090E008957C3FD9F76230C8F78630B8F78D
:1035F00040E0B1CFCF92DF92FF920F931F93CF9312
:10360000DF936C0100910C0880910B08082BC5E03A
:10361000D0E010E0C8010C2E02C0959587950A9461
:10362000E2F780FD0CC02197A8F7F12C8F2DDF91D8
:10363000CF911F910F91FF90DF90CF900895FC2EB6
:10364000B6018C2FBCDF0E942D08019761F3EECFED
:103650001F93CF93DF93FC012581C081D181CE01DF
:10366000211579F0611569F0C5DF182F682FCE019B
:103670000E947D06BE01812FA2DFDF91CF911F91B5
:1036800008950E949606182FF5CFCF93DF93EC0193
:10369000B1DFBE0194DF0E942D08DF91CF91089524
:1036A000FC012481211599F080819181EEDF282F82
:1036B00092959F70963099F060F4925F9F7092306F
:1036C00030F4203FB1F038F481E0283E38F080E05B
:1036D00008959A5FF3CF81E0243FC9F7089591E000
:1036E000213F09F090E081E0283E08F080E0892B3E
:1036F000089581E00895673D71058105910528F4DD
:10370000CB01875D9C4F0C94BA3480E00895CF9232
:10371000DF92EF92FF92CF93DF93EC01C880D980C4
:10372000EA80FB80B601C701E6DF9FEFC91AD90A1C
:10373000E90AF90AC882D982EA82FB82DF91CF9135
:10374000FF90EF90DF90CF90089585E290E00E9487
:10375000BA34863269F486E290E00E94BA34883046
:1037600039F487E290E00E94BA3491E0843009F0A5
:1037700090E0892F8170089580E090E00E94C2342B
:10378000833E9E4F09F4E1CF80E0089548E050E089
:1037900067E170E084E897E00E94C7341092E90482
:1037A000089581E18093840780919B0190919C0111
:1037B000A0919D018093850790938607A09387072A
:1037C0008FE7809388078FEF80938907DFCFCF92B1
:1037D000DF92EF92FF920E94A30FAB01BC014093D6
:1037E000E0045093E1048093E2047093E304809139
:1037F000E40490910D01923049F1F0F4911123C04D
:10380000109210014093E5045093E6046093E7049E
:103810007093E80480911E07811108C0809184078D
:10382000982F937019F086958695982F9093E404BD
:1038300081E080930D0102C0933099F0FF90EF90EA
:10384000DF90CF9008950E940D0BF8CF80930F0169
:1038500080918407837080930E010E94281283E078
:10386000E8CF8091E904811191DFC090E504D09008
:10387000E604E090E704F090E8048091B507811534
:1038800071F00E94970F6C197D098E099F096530B0
:1038900071058105910590F210920D01CFCF0E9424
:1038A000A30FF1CFA0E1B0E0E8E5FCE10C943F34D8
:1038B000FE013196DF0180E11D928A95E9F70EE065
:1038C00010E099E2A92E93E0B92E612C712C23010E
:1038D0004A189E2E8F2E6201730181E14816510411
:1038E000610471041CF080E1C82ED12CA601B50141
:1038F000892D982D0E94C734AC0CBD1C0D2C000CDA
:1039000000084C185D08600870080150104019F755
:103910006096E0E10C945B346FEF85E290E00E94EA
:10392000D6346FEF86E290E00E94D6346FEF87E2E4
:1039300090E00E94D63460E088E290E00E94D634A5
:103940000E941B13AFDF66E285E290E00E94D6344E
:1039500068E086E290E00E94D63464E087E290E07E
:103960000C94D63463EE7EEF80E090E00E94F03459
:1039700060E082E090E00E94D63481E080930B0802
:1039800061E083E090E00E94D63460E074E184E07E
:1039900090E00E94F03405DFBFDF60E070E0AB0133
:1039A0008FE090E00E94E83460E070E0AB0183E1DA
:1039B00090E00E94E834EACEAB0124E630E0BC019E
:1039C00088E70E94F2319C0181E0232B09F080E01E
:1039D00008958091EF068115F1F00E94970FDC01A8
:1039E000CB01805A9541AF4FBF4F8093F006909323
:1039F000F106A093F206B093F306809119078111A6
:103A00000AC062E070E08CE596E0D6DF811519F01F
:103A100081E08093190708958091EF06811561F088
:103A200080911907811541F062E070E08AE596E027
:103A3000C3DF81111092190708951F921FB61F92BC
:103A400011248F939F93AF93BF938091F6068111BA
:103A500013C08091C7039091C803A091C903B0918E
:103A6000CA034196A11DB11D8093C7039093C8035B
:103A7000A093C903B093CA03BF91AF919F918F9157
:103A80001F901FBE1F9018952FB7F8948091C70301
:103A90009091C803A091C903B091CA032FBF0895A4
:103AA000CF93DF93EC01F0DF8C1B9D0BDF91CF9167
:103AB0000895AFE0B0E0EFE5FDE10C944434FE0181
:103AC0003196DF018AE01D928A95E9F783E1C82EDD
:103AD00083E0D82E7F01AE2E9F2C0EE113E0F6017D
:103AE00081916F018F3F09F43DC0F894E82FE29572
:103AF000EF70F0E021A18F7041E001C0440F8A9582
:103B0000EAF7922F942B91A392A1842F8095892379
:103B100082A3789400C0E8E1F3E031E0B12C219178
:103B20002F3F79F0A22FA295AF70A05EB0E08C91EC
:103B300090E02F7002C0959587952A95E2F780FF57
:103B4000B7C080E0B82A330F0E171F0741F7F60100
:103B500082918F3F11F00E941B0980EA8A95F1F74C
:103B6000F701B0828FEFE81AF80A88E1C81683E0FF
:103B7000D80609F0B4CF4AE050E06A2D792D8BEADF
:103B800097E00E949434009749F02AE0EA2DF92D3D
:103B9000ABEAB7E001900D922A95E1F70091AA07F0
:103BA00010E00056184F892B09F484C081E08093FF
:103BB0009F076ADF80939D0790939E078091B507CA
:103BC000811509F4CEC07E018BE0E80EF11CF701EF
:103BD00085E011928A95E9F7809198078A3008F07C
:103BE0008CC044EF58E1B701C8010E94F51181155E
:103BF00009F4A6C04FEF59E1B701C8010E94F511C1
:103C0000811509F49DC04FE159E1B701C8010E9437
:103C1000F511811509F494C040E658E1B701C801D7
:103C20000E94F511811509F48BC04EE959E1B701E5
:103C3000C8010E94F511811509F482C04DE05AE1D6
:103C4000B701C8010E94F511811509F479C045E258
:103C50005AE1B701C8010E94F511811509F470C03D
:103C600043EC59E1B701C8010E94F511811509F42F
:103C700067C048E45AE1B701C8010E94F5118115F7
:103C800009F45EC01092980780919C0790E045E08F
:103C900050E0B7018056984F0E94943421E0209361
:103CA0009B07892B09F03FC02F96EBE00C94603402
:103CB000832F48CF80919F07811509F47FCFE09033
:103CC0009D07F0909E07E0DE8E199F09059708F486
:103CD00075CF45E050E06BEA77E0C8010E9494346C
:103CE000892B41F085E0EBEAF7E0D80101900D92D5
:103CF0008A95E1F710929F0761CFC0909907D09005
:103D00009A07C2DE8C199D09843F914008F069CF63
:103D100080919B07811541F2F70185E011928A9508
:103D2000E9F710929B07A0919C07B0E0A056B84F0E
:103D300085E0FE013B9601900D928A95E1F7B4CFA4
:103D4000809198078F3F31F49FDE8093990790937D
:103D50009A07DECF8F5F809398078A3008F494CF5C
:103D6000F3CFE0909C07F12CC7018056984F7C015F
:103D700085E0F801A7E4B7E001900D928A95E1F79C
:103D800065E070E087E497E00E946D0E809346073F
:103D900085E0ECE4F7E0D70101900D928A95E1F718
:103DA00088E0E7E7F7E0A2E5B7E001900D928A9599
:103DB000E1F768E070E082E597E00E946D0E809385
:103DC0005107C0905A07D0905B07E0905C07F090D5
:103DD0005D0780917F0790918007A0918107B09146
:103DE0008207C816D906EA06FB06B1F0C0927F0723
:103DF000D0928007E0928107F09282070E94970F8D
:103E0000C61AD70AE80AF90AC092B707D092B807CB
:103E1000E092B907F092BA0780915E0780930C0890
:103E200080915F0780930B088091600780938307E0
:103E300088E0E1E6F7E0A4E8B7E001900D928A950A
:103E4000E1F7809169070E94B40C80916A0781159F
:103E500091F1BFDD8091730790917407A091750770
:103E6000B091760740916F0750917007609171078C
:103E70007091720700916B0710916C0720916D078C
:103E800030916E070093940710939507209396073F
:103E90003093970740939007509391076093920750
:103EA0007093930780938C0790938D07A0938E0750
:103EB000B0938F07F9CEB0DDCDCF2F923F924F92C6
:103EC0005F926F927F929F92AF92BF92CF92DF925A
:103ED000EF92FF920F931F93CF93DF938091EF06A2
:103EE000811509F47BC0C091DE04D091DF04CCDDE4
:103EF0008C1B9D0B819708F450C0C6DD8093DE04B7
:103F00009093DF0480E00E94B30D80910C080E9422
:103F10001A118091B607811509F48DC080E00E94C6
:103F2000B30D60E670E08AE795E00E94C40D83E07F
:103F30000E94B30DE091EC04F091ED049F012E5E20
:103F40003440BF016E5A7340613082E0780710F050
:103F500060E072E04091EA045091EB04A6E6B8E01C
:103F6000D1E0ED2EF12C2617370708F449C0409315
:103F7000EA045093EB048DE00E94B30D60E470E01E
:103F80008AE196E00E94C40D8FE00E94B30D60E2CA
:103F900070E08AE194E00E94C40D8091EA0490915F
:103FA000EB04892B09F068C0809119078115B1F0E5
:103FB0000E94970FC091F006D091F106E091F206B1
:103FC000F091F306DC01CB018C1B9D0BAE0BBF0BFC
:103FD0008F3F9F4FAF4FBF4708F41EDDDF91CF915A
:103FE0001F910F91FF90EF90DF90CF90BF90AF9017
:103FF0009F907F906F905F904F903F902F9008958B
:104000008D9191918917A1F08F0101501109E8015B
:104010008883C901C5E096958795CA95E1F7E701C0
:1040200002C0CC0FDD1F8A95E2F7CE014C2B592B35
:104030002F5F3F4F98CF0E94D40ECAEDD4E081FD90
:1040400002C0CAE3D4E080E00E94B30D60E670E0F5
:104050008AE795E00E94C40D84E00E94B30D60EAF7
:1040600070E0CE010E94C40D8DE00E94B30D60E4AB
:1040700070E08AED95E08FCF8091EF06811509F40D
:1040800093CF8091EE0681118FCFA3DCC0E0D1E108
:104090002091EA043091EB042115310509F484CF15
:1040A000D15009F481CF41E050E001C0CF5F8C2FA7
:1040B00090E07A010C2E02C0EE0CFF1C0A94E2F78D
:1040C000B70162237323672B89F32091F50620FD46
:1040D00043C09695879596958795482F282F9C2FB6
:1040E0009295990F9076392F315E842F9093060127
:1040F000809309013093070120930A0124E630E000
:1041000047E050E064E071E088E70E94A831892B25
:1041100009F04ACF80E2C89FA00111248091F506E2
:1041200080FD23C042515B4F04E610E020E230E006
:1041300060E488E70E943832892B09F035CFE0949B
:10414000F0948091EA049091EB04E822F922E09245
:10415000EA04F092EB049CCF9C2F990F990F990FD2
:10416000392F395F80E023E0C1CFEEEBF4E080E24D
:1041700011928A95E9F731EB632E31E0732E0DEA47
:1041800011E065EB71E0D301ED913D01D8018D9116
:104190008D01282F240F352F311D1901F0E0E25435
:1041A000FB4F80E090E027E0A22EA81ABB24B39436
:1041B000082E01C0BB0C0A94EAF7910122513B4F33
:1041C0002901C12CD201DD902D01DB202A2D2C19D3
:1041D000277030E0AD2D022E01C0AA0F0A94EAF735
:1041E0009A2E3195219531092770332701C0D69435
:1041F0002A95EAF79D282081922A9082C3942C2D3B
:10420000283001F7019631968830910561F66615E0
:10421000770509F0B8CF04E610E020E24EEB54E059
:1042200087CFFF920F931F93CF93DF93C62FD42F87
:10423000F22E8115A9F06093060826DC8093E40332
:104240009093E50381E0C1FD84E0C0FD880FC2FDCD
:1042500082950E94DC13CDB7DEB7E5E00C9466349E
:1042600080910608681333C00091E4031091E503C0
:104270000BDC801B910B883C910548F51D2F105ECF
:10428000CD17A1F0C77001E0802F01C0880FCA953B
:10429000EAF70E94EE13183048F48D2F877001C0A2
:1042A000000F8A95EAF7802F0E94DC136AE070E025
:1042B0008F2D0E94D11481E0D1FD84E0D0FD880FC4
:1042C000D2FD8295183038F60E94EE13C4CF81E0FB
:1042D000C1FD84E0C0FD880FC2FD8295F5CFA4E04A
:1042E000B0E0E5E7F1E20C9442347C01FC0184810A
:1042F000811509F426C161E0C701AAD96C01F70153
:1043000085818115D1F000910208109103080115F3
:10431000110599F0C016D10689F020E9A22E21E0FE
:10432000B22E011511F0A12CB12C60E0802F0E945B
:10433000850EFC01892B09F04EC08601F70195819D
:1043400002348EE7180709F49FC008F054C0003407
:104350008EE7180709F45EC001348EE7180709F4E8
:1043600078C0F7018581811509F46FC1980137572D
:104370002038310508F069C1003108F0D3C066ED7E
:1043800070E080E090E0B7D98111CCC0A12CB12CB5
:10439000450101118AC089829A82AB82BC828E015A
:1043A0000F5F1F4FC801B3D9B02EA12E813008F482
:1043B000B9C009F0E1C0C801AAD9813009F087C0AD
:1043C000C801A5D960E570E0893311F06AE070E0BA
:1043D0000E94D11482C0858184608583C082D1828D
:1043E000BF01C5010E94E1171092100861E0C701EA
:1043F0002FD98C01A3CF03348EE7180709F0B1CF72
:1044000080910F088170911509F44BC081112FC064
:104410008DE40DC080910F088170911569F08115B0
:1044200049F084E00E94DC070E94DC1380E50E94D2
:10443000FE1397CF81E0F6CF811549F084E00E940A
:10444000DC070E94EE1380E50E9482148ACF81E08F
:10445000F6CF80910F088170911559F0811539F0D0
:1044600084E00E94DC070E94DC138FE4E0CF81E04F
:10447000F8CF811539F084E00E94DC070E94EE132A
:104480008FE4E2CF81E0F8CF80910F088170911521
:1044900021F08111CFCF8AE4CACF8111D8CF8AE42D
:1044A000D3CF8111EFCF8DE4CFCF87ED8816910464
:1044B000A104B104B9F1B401C5011DD99FEF891A56
:1044C000990AA90AB90A8111F0CF015062CF82304E
:1044D00059F4C8011CD90E94FE138FE39CE901978F
:1044E000F1F700C000005ECF833029F4C8010FD976
:1044F0000E948214F2CF843069F4C80108D9C12C1B
:10450000D12C282F2053330B2A303105F0F0C11461
:10451000D10441F5EFE3FCE93197F1F700C0000069
:10452000811140CF80910D08877059F0F701858186
:10453000811539F080910F0882FF03C082E00E944C
:10454000F4062496EDE00C945E344AE04C9DC001E4
:104550004D9D900D1124280F391F69018B2D9A2D27
:10456000D6D8CFCFEFE9FFE03197F1F700C00000D8
:1045700091E0C91AD108CBCFE82FF0E0E055F84F11
:104580009491792E282F26952695269530E0F901CD
:10459000E056F84FC4908770D12C082E02C0D594F5
:1045A000C7940A94E2F7F901E057F84FA490B12CB0
:1045B000082E02C0B594A7940A94E2F72058384F09
:1045C000F9018490912C02C0959487948A95E2F722
:1045D000C0FE09C081EE0E94FE138FE39CE90197A3
:1045E000F1F700C00000A0FE09C086EE0E94FE1395
:1045F0008FE39CE90197F1F700C000006AE070E0EA
:10460000872D0E94D1148FE39CE90197F1F700C038
:104610000000A0FE09C086EE0E9482148FE39CE990
:104620000197F1F700C00000C0FE09C081EE0E94B2
:1046300082148FE39CE90197F1F700C0000080FE2F
:10464000B1CE6AE070E08CE2C3CE312F375509F06D
:104650007EC0A02EB12C011165CF682F80E00E9492
:10466000850E6C01892B09F45DCFF7018581F60178
:10467000958180FB90F99583811509F448C004DA8F
:104680008093040890930508F60182818F5F8283EE
:104690008091100890910808892B838380910908E4
:1046A00084834091900150919101609198017091A3
:1046B0009901C6010E94CE0EF601858181FD03C0DD
:1046C000A12C97E5B92EA0920208B0920308F70139
:1046D0009581911509F450C410920608980130573D
:1046E0002332310508F035C484E090E00E94C234E2
:1046F00080930E0890930F08F801E150F047E232E2
:10470000F10508F04BC0E85FFA4C0C9487344091F7
:104710009601509197016091980170919901C6019D
:104720000E94CE0EF601858181FFD1CFB60180E9CE
:1047300091E00E94C41780910208909103088115AE
:10474000974529F61092020810920308C0CFF8018D
:10475000E851FC47E730F10508F0B9CFE65DFA4CC7
:104760000C94873426E241EE61EE5BDDDBCE27E27E
:1047700045EE65EEFACF26E241EE60EEF6CF27E297
:1047800045EE64EEF2CF26E241EE62EEEECF27E296
:1047900045EE66EEEACF28E241E0EBCF80910E08CD
:1047A000816080930E0860910E0870910F0884E07C
:1047B00090E00E94F0340E94E514B4CE80910F087E
:1047C000886080930F08EFCF80910E088260E9CF58
:1047D00080910E088460E5CF80910E088860E1CF5B
:1047E00080910F088160EDCF80910F088260E9CF42
:1047F00080910E088061D5CF80910E088062D1CF64
:1048000080910E088064CDCF0E94E51480910E083F
:104810008068C7CF80910E088C60C3CF80910F084D
:104820008360CFCF80910E088E7FBBCF80910F0821
:10483000877FC7CF80910E088D7FB3CF80910E0800
:104840008B7FAFCF80910E08877FABCF80910F0811
:104850008E7FB7CF80910F088D7FB3CF80910E08E8
:104860008F7E9FCF80910E088F7D9BCF80910E0809
:104870008F7B97CF0E94E51480910E088F7791CFA0
:1048800080910E08837F8DCF80910F088C7F99CF08
:1048900090910E08892F8B7F92FF8460877F92FF13
:1048A00088607FCF80910F08982F909590FB80F9BA
:1048B00090FB81F986CF90910E08892F8F7B96FF10
:1048C00080646FCF0E94E51490910E08892F97FBAA
:1048D00087F9805866CF61E08EE090E00E94D63480
:1048E00062CF60E0F9CF90910E08892F8F7E94FF00
:1048F000806157CF90910E08892F8E7F90FF816045
:1049000050CF90910F08892F877F93FF886059CFF0
:104910008A7A91E0811101C090E09093070881119B
:1049200006C089E20E94380F0E948613FBCD85E302
:10493000F9CF85E32BC381E00E94CC0CF3CD811528
:1049400079F10E94130DEECD811579F10E94350D9C
:10495000E9CD811579F10E944A0DE4CD811579F1F7
:104960000E94620DDFCD811579F10E94780DDACDBC
:10497000809108088272F801E054F847EF30F105A1
:1049800080F5EF5CFA4C0C9487340E94D50C81E0E2
:104990000E946D0AC7CD0E94E20CF9CF811589F201
:1049A0000E94090DBFCD811589F20E942C0DBACD50
:1049B000811589F20E943E0DB5CD811589F20E94C4
:1049C000560DB0CD811589F20E946E0DABCD8115CB
:1049D00029F00E94990DA6CD8115D9F30E94820D70
:1049E000A1CD07378CE71807F1F008378CE71807D7
:1049F00029F19801205E32452032310520F59111D0
:104A000034C00F7181E090E002C0880F991F0A95B1
:104A1000E2F78C01682F83E090E00E94D634802F6B
:104A20000E940E067FCD81E0911551F00E94140680
:104A300043E062E081E00E94AD0674CD82E0F4CFF5
:104A40000E941D06F5CF911581F10B358CE71807F3
:104A500011F10C358CE7180799F00A358CE7180727
:104A6000C1F001308CE71807F1F003308CE718072C
:104A7000A1F001151C47C9F40E94E5140E94BE0F65
:104A800080910F08002482FF0394802D0E94AD12B4
:104A900049CD81E0FBCF80E0F9CF6FEF7FEF80E081
:104AA00090E00E94F0340E940215F701008111810C
:104AB000911509F45BC0C8010E94FA1AD82E682F1C
:104AC000C8010E947D06B8018D2D0E94DF1A0E9448
:104AD0002D08182FA92EF701B580D680D2948FE02B
:104AE000D82280910D08877001F1CB2CB114F1F020
:104AF000892F807F803461F0812F805E8830A8F01C
:104B0000892F807E803221F4123078F0D11469F040
:104B100080910F0882FF09C082E00E94F406809114
:104B20000D088770CC24C3948111C12C8A2D8295E5
:104B30008F70883009F40EC1C0F58430E0F4823003
:104B400008F444C00A2D0F708A2D807F803211F046
:104B50000295007F113008F472C009F4BBC0B11493
:104B600009F4C6C0D11409F488C048C0C8010E9425
:104B70009606D82EA8CF09F4D1C0C11409F419C1E2
:104B800080910D0880FD15C1F701158286958695E7
:104B900086950E941406C701A2DB80910D088695B8
:104BA000869586950E941D0604C1893009F44DC181
:104BB0008A5F8F70823008F7123F09F058C18A2D42
:104BC0008F71B11051C10E941406F1C00A2D0F70EF
:104BD0008A2D803110F00295007FB114B9F00115D3
:104BE00069F0812F805E883010F0111109C080912A
:104BF0000808802B809308080E948613812F2FC0FD
:104C000080911008802B80931008F6CF812F0E948E
:104C10008214011509F4B1CF812F805E883010F025
:104C2000111104C0802F0E94310706C000958091A9
:104C300010088023809310080E9486139ECF8091D5
:104C40000F0882FD16C0B11469F0011539F080918A
:104C50000808802B809308080E94861380E00E9439
:104C6000FE138BCF80E00E948214011509F485CFDA
:104C7000D9CFB114A9F0D11004C0802F0E94DC1349
:104C80007CCF8D2D813009F078CF80910908902F4D
:104C90009823091709F471CF802B809309086DCFF1
:104CA000D1106BCF802F0E94EE1390910908802FB6
:104CB000892329F0802F809589238093090880918A
:104CC0000A08902F982309F458CF009508230093E1
:104CD0000A0853CF8D2DB11421F0863008F04DCF46
:104CE000CCCF853008F049CF802F0E94EE1345CFFE
:104CF000D114D1F3193369F48FEF97EE23E081508B
:104D000090402040E1F700C00000812F0E948214F3
:104D100034CF8FE39CE90197F1F7F5CF8A2D869583
:104D200086958370813060F009F027CF812F9A2D0E
:104D30009370B11002C080E090E00E94110F1DCF6F
:104D4000812F9A2D9370B11002C080E090E00E94F4
:104D5000EA0E13CF8A2D8370E1F5B11028C0812FA0
:104D6000829586958770880F880F412F4F70082E87
:104D700001C0440F0A94EAF7212F207114FF06C0E6
:104D80002FE001C0220F8A95EAF720958A2D86959B
:104D900086958370982F8230A1F08330B9F080918E
:104DA0000B08913059F0242B82230E940E060E949A
:104DB000D40E60E0C7010E94281BC3CB842B822B3A
:104DC000F4CF242B80910B088227EFCF822F842BE6
:104DD000ECCFB11459F1A0FEEACF812F82958695D0
:104DE0008770880F880F412F4F70082E01C0440F25
:104DF0000A94EAF7212F207114FF06C02FE001C0AA
:104E0000220F8A95EAF720958A2D869586958370DC
:104E1000982F823091F08330A9F080910C08913066
:104E200049F0242B82230E941106C1CF823008F45E
:104E3000BECFD3CF842B822BF6CF242B80910C08AE
:104E40008227F1CF822F842BEECF8A2D8F70082FEF
:104E5000B11431F00E941406812F0E94DC13A7CFF9
:104E6000812F0E94EE13802F0E941D06A0CF70F4A8
:104E7000103FC9F0113F91F0B11409F451C0D114A1
:104E800009F44BC0812F0E94FE1391CF133FF9F01C
:104E9000143F91F790910F0892FD26C08A2D8F71D3
:104EA000B11411F390CE8D2DB11479F0853008F046
:104EB0007ECF8A2D8F71282F81E001C0880F2A951F
:104EC000EAF790910C088927AECF8630F0CF80E0CA
:104ED000B11409F4A8CF8A2D8F71982F81E001C0F9
:104EE000880F9A95EAF79FCFB11461F08A2D8F71E0
:104EF00092FF69CE982F990F990F990F9360909315
:104F00000D0861CE81E00E94F4068D2D823008F4F8
:104F10004ECF82E00E94F4064ACF8A2D8F7153CE85
:104F2000D114A1F0193369F48FEF97EE23E081508B
:104F300090402040E1F700C00000812F0E948214C1
:104F400036CF8FE39CE90197F1F7F5CF8A2D8F716A
:104F50008BCF8091080806312CE7120709F4D8CCD2
:104F60008272F801E052F847EB30F10508F039CDD4
:104F7000E05CFA4C0C94873406318CE7180709F092
:104F8000F7CC809107088111D4CC89E20E946C0F84
:104F9000CBCC80915108803170F4809150088115FC
:104FA00051F0E09112082091110830914C08409185
:104FB0004B082E1301C00895BF0187E0E89FF00160
:104FC0001124DF01AD5EB74F14968C9114978115B3
:104FD00051F111968C911197831325C08C918413F4
:104FE00022C015968C91159781111DC012968D9136
:104FF0009D91A0914D08B0914E088A1B9B0B883C57
:10500000910588F4809151088F70806180935108D8
:10501000E75EF74F80818F70806180838BE498E03A
:105020005ED90C94EA066F5F7F4FFB01E770C1CF3A
:10503000ADE0B0E0EEE1F8E20C9442348C0186E0A1
:10504000F801DE01189601900D928A95E1F7F801BA
:10505000F58084819BE4892E98E0992E70904F080A
:10506000711017C0811591F0F11409F40EC1C80137
:105070000E94501B811509F408C187E0F801ABE4D8
:10508000B8E001900D928A95E1F783DFFF24F39455
:1050900055C0D080A280B380C090500820914D08A8
:1050A00030914E08A501421B530BC11409F4BDC039
:1050B000483C510508F076C0811541F380914C08B9
:1050C0009180E09051089E2D903108F057C09812C1
:1050D00014C080914B088D1110C0F11049C08E2D65
:1050E0008F708061809351088BE498E0F8D88091AC
:1050F0005108F8018683F12C21C0F11039C040E03D
:10510000692D8D2D0E94CB0640E0692D8D2D0E94CA
:10511000CB06F82E8111EFCF888599850E94451B1B
:10512000292F22952F70903470F49F70223098F0C0
:105130009115A9F0F8019681903188F48F2D2D9664
:10514000EDE00C945E342A5F2F70223060F0C801CD
:10515000C6D8FC2CF3CF911511F0811579F3805E40
:10516000883060F3F4CF803F48F3815F8330F9CF1C
:1051700080915108816080935108BDCF981237C04B
:1051800080914B088D1133C0F11031C0E682C80107
:10519000A6D887E0F801ABE4B8E001900D928A95BB
:1051A000E1F774CFE09051089E2D903148F48BE4E4
:1051B00098E095D8F40187E011928A95E9F79BCFA2
:1051C000811509F463CF90914C08818198130FC029
:1051D00080914B088D110BC0F11009C0E682C80107
:1051E0007ED8F40187E011928A95E9F74FCFC80184
:1051F0000E94501B811509F448C0F11409F445C000
:105200008E2D803208F439CF80914B0890914C0854
:1052100089839A83AB82BC827D821E8280915108F1
:105220008F83CE0101965BD828CF483C510508F00A
:10523000C1CF811509F42ACFF11439F190914C08AE
:105240008181981318C080914B088D1114C08091F2
:10525000510880FD9ECF803108F49BCF8683807FEC
:10526000803F09F494CF8681982F907F905F8F7054
:10527000892B86838CCFC8010E94501B8111FDCEE3
:1052800080915108816080935108C80128D8FECED2
:10529000ABE1B0E0EEE4F9E20C944B344E8B5F8B63
:1052A000688F798F8A8F192F9B8F91111092100818
:1052B0001D8A86E0FE017696DE011F9601900D9212
:1052C0008A95E1F70A8D011561F00B8B1C8B61E06B
:1052D000CE010F960E94281B61E0CE010F960E941E
:1052E000281B0B8B1C8B87E0FE013F96DE01189676
:1052F00001900D928A95E1F7CE01089699DE811111
:105300002EC0209111083091120887E0AE01485F4D
:105310005F4FFA0147505109DA0101900D928A95C9
:10532000E1F78C858115D9F0822F90E08395877005
:1053300090E0AC0134171506E1F097E0929FD001A0
:105340001124AD5EB74F9E012F5F3F4FF9010190D1
:105350000D929A95E1F7409311080E94EA06809118
:10536000120890911108891311C06B96E4E00C9417
:1053700067340E94E5141092110810921208EBE4B1
:10538000F8E087E011928A95E9F7E9CF27E0829F5C
:10539000C00111248D5E974F4BDE811531F3809152
:1053A0001208909113080196877080931208D7CF46
:1053B000A6E0B0E0EEEDF9E20C944B340E94441DFF
:1053C0008C018091BB079091BC078017910771F009
:1053D00019821A820E94441DBC0149815A8180E0D1
:1053E00090E056DF0093BB071093BC072696E4E0DD
:1053F0000C946734ACE0B0E0E0E0FAE20C9448349E
:1054000080E09CEFE92E2DEFD22E90917A0720912B
:105410007907291709F448C0E92FF0E0E558F84F5B
:10542000F0800F2D0F779F5F937090937A07809194
:1054300078078F5F80937807F7FC06C00F83E886B4
:105440000E94441D13E005C00F83D8860E94441DAE
:1054500012E0BC0189879A871B8781E08C874F8186
:105460005885812F91E014DF8FE39CE90197F1F7D4
:1054700000C000000983F7FE15C0DA820E94441DB7
:10548000BC018B839C831D831E8249815A81812F9D
:1054900090E0FEDE8FE39CE90197F1F700C0000089
:1054A00081E0B3CFEA82EACF2C96E7E00C94643433
:1054B000CDB7DEB7A0970FB6F894DEBF0FBECDBF55
:1054C00085B7806885BF85B7806885BF84B7877FCB
:1054D00084BF0FB6F894A89580916000886180938E
:1054E0006000109260000FBE80E890E00FB6F89464
:1054F00080936100909361000FBE81E080938F01E3
:1055000089E199E080938A0390938B030E94FC10B9
:105510000E94AD108091E20084608093E200789454
:1055200080911407811599F08091E9001091EC00A9
:105530008F7010FB112717F9182B1092E90080913A
:10554000E80083FD0E940E151F701093E90082E0B1
:1055500084BD93E095BD9AEF97BD80936E00109245
:10556000B7071092B8071092B9071092BA070E94B5
:10557000A51B811102C00E948C1C8091D800806103
:105580008093D8008AE18A95F1F700C08091D90014
:10559000182F117080FD04C00E94FC101092140797
:1055A0001093B5070E94BC1B811102C00E94B21C5F
:1055B0008EE090E00E94BA34811529F060E08EE020
:1055C00090E00E94D6348EE090E00E94BA3491E0E0
:1055D000811101C090E09093B607909315018091DE
:1055E000B5078111E7D7E7E7F7E088E011928A95E0
:1055F000E9F78091B60791E0282F292720930F071C
:1056000090931207811106C084EF8093170185EFF4
:105610008093160160E080E00E94230E61E080E04C
:105620000E94230E8FE891E00197F1F700C000007F
:1056300010E080911207181708F462C08091B60735
:1056400090E0811101C095E09093AA0785E0891B45
:1056500080939C07E3E1EE2EE3E0FE2E08E113E0E9
:10566000F70181917F018F3F11F00E941B090E15F8
:105670001F05B1F708E113E0F80181918F018F3F19
:1056800011F00E941B0983E00E311807A9F7E0EA28
:10569000F7E08AE011928A95E9F7EBEAF7E08AE011
:1056A00011928A95E9F70E94BC1B811102C00E94E9
:1056B000B21C82E090E00E94BA348093020784E03A
:1056C00090E00E94C23480930E0890930F080E94CD
:1056D000591D8FEF96E721E0815090402040E1F77F
:1056E00000C000000E94591D8091A00780FF1AC0D1
:1056F0006FEF7FEF80E090E00E94F0340E94BE0FD9
:1057000060E0812F0E94430E082F61E0812F0E94EC
:10571000430EE12FF0E0E05FF84F880F802B80838D
:105720001F5F87CF83E090E00E94BA340E940E068C
:105730000E94600E81E08093E90448E050E067E158
:1057400070E084E897E00E94AA341092E904809106
:105750008407843010F40E94D11B83E08093F50607
:1057600080E28093F406C1D56BE070E085E797E0B6
:105770000E94DC1C8115E9F18091F50665E070E07E
:1057800081FD07C180E797E00E94DC1C811589F14B
:105790006DE070E08EE597E00E94DC1C811549F118
:1057A0000E94970FDC01CB01805A9541AF4FBF4F4C
:1057B0008093F0069093F106A093F206B093F3065F
:1057C000EEEEF4E0DF0180E092E01D920197E9F750
:1057D000E093EC04F093ED048FEF9FEF8093EA04E5
:1057E0009093EB0481E08093EF0680931907109269
:1057F000EE068091B507811101C0DFD68DEE92E0F3
:10580000809364089093650884E080936308ADEE0C
:10581000B2E020E013968C911397811501F12830A6
:10582000F0F4822F90E0FC01EE0FFF1FEE5AF74FCD
:105830008F01009761F0F801529142918F01FA01B6
:10584000348114966C911497631708F4A5C0880FDF
:10585000991F8E5A974FFC01A083B1832F5F159635
:1058600083E0A130B807B1F62093620880910C085C
:105870000E941A1188E191E08093DD079093DE0782
:1058800051E0A52EB12C8091140700E110E442E113
:10589000F42E853009F4E1C00E94591D33E0C32E77
:1058A00037E0D32E80EA97E01C012DE037E0FC01C1
:1058B000D6019D9180812A173B0709F4DBC0319600
:1058C0009817B9F34090B50728EFE22E26E0F22EA4
:1058D000912CF10181901F01F60181916F018815D2
:1058E00009F442C08825582E00E010E07724739414
:1058F000852D872189F1682C67204114F9F0F70183
:10590000808190E09501002E01C0220F0A94EAF7F1
:105910008223892B99F409839A820E94441D8B83E8
:105920009C8381E08D8391E0611001C090E09E83B3
:1059300049815A816B817C818D81AADC61100CC008
:105940008A2D002E01C0880F0A94EAF7982F9095AF
:10595000F701808189238083770C0F5F1F4F06300A
:10596000110531F6F601829293948FEFE81AF80A46
:10597000892D8A3009F0ADCF0E94A30F6093940760
:10598000709395078093960790939707DD24D3949F
:1059900075C08BE697E0F8CE0197F80142835383F8
:1059A00048CF80911407843051F10E94E71B81E0B9
:1059B0000E94B40C0E940C1D1092F60688E190E043
:1059C0000FB6F894A895809360000FBE1093600006
:1059D00083B7817F846083BF83B7816083BF7894FE
:1059E000889583B78E7F83BF0FB6F894A895809172
:1059F0006000886180936000109260000FBE0E947A
:105A0000591DE0EAF7E0A8EFB6E080E021912D9380
:105A100091E0211101C090E0892B2AEA37E02E178E
:105A20003F07A1F78115C9F08091F7068115A9F00C
:105A300009BDF9BC09B400FEFDCF8091D8008F7D6F
:105A40008093D8008091E00082608093E000809194
:105A5000E00081FDFCCF0E94E514809114078530A1
:105A600009F49FCF0E94E5140E94D40E80E00E94AA
:105A7000B40C12CF981326CF9BDCD12C8091B507A4
:105A8000811541F1009102081091030801151105DB
:105A900009F1E0900408F09005080E94441D8E1959
:105AA0009F09893C9105B0F090E9E92E91E0F92E2B
:105AB000011511F0E12CF12C60E0802F0E94850E81
:105AC000009741F0FC01258122FD04C0BC01C70103
:105AD0000E94E1170E94E71BF090B507F11411F046
:105AE00089DCF82E80913307811551F0109233072D
:105AF0008091790780937A07809177078093780760
:105B0000E12C38C061E08E2D0E94430E182F60E01A
:105B10008E2D0E94430E110F812B0E2D10E0D80107
:105B2000A05FB84FEC919E2F9370891711F1EE0F83
:105B3000EE0FE82BEC9380910F078E0DEF70F0E0E5
:105B4000EF5FFC4F035F184FC080F8019081C90ED2
:105B50009C2D60E092301CF49F3F1CF461E00E9499
:105B6000030E8C2DCC0C990B62E070E0BDD6F801D1
:105B70008083E39480911207E81620F28091B507A4
:105B8000811511F037DCF82AF11479F00E94A30F87
:105B90006093900770939107809392079093930777
:105BA0000E945D1F0E94E91C04C00E945D1FD1106D
:105BB000F9CF0E94D40E90911307891721F080939A
:105BC00013070E94970F80911407843009F05BCE71
:105BD00083E08093E9008091E80082FF54CE8091B9
:105BE000E80090E085FF05C00E947C10811591F0CF
:105BF00091E08091E8008B778093E800911509F49B
:105C000042CE8981E82FE150E53168F5F0E0E55BAF
:105C1000FA4C7DC680E2E82EF12C8E010F5F1F4FFB
:105C20008091E80085FD0AC08091E8008B77809321
:105C3000E8000E947C10811599F3DACF8091F10081
:105C4000F801808381E0E81AF10891F2E7CF1A8227
:105C50008CE08B8319C08A81833081F138F48130E4
:105C600029F1823051F08FEF89830EC08430D9F74B
:105C70001B821C821D821E8207C088E290E07AD6B9
:105C80001B821C821D828E83E091DD07F091DE076E
:105C9000309709F4F8CD0284F385E02D309709F4AC
:105CA000F2CD60E2CE0101960995EDCD0E94970FED
:105CB00034D66B837C838D839E83E6CF8B8190E08B
:105CC000FE0134968A309105FCF611920196FACFC6
:105CD0008A81823031F0853031F680E00E94CC0C30
:105CE000D3CF6B817C818D819E8117D688E290E035
:105CF0005DD6CACF4C816B818A810E94811A982718
:105D0000892798278D839E83BFCF2D813E8132279F
:105D1000232732274C816B818A810E94C412B4CF21
:105D20000E941B13B1CF9A81933009F09CCF883029
:105D300009F439C0893009F462C08B81833061F184
:105D400058F4813091F0823009F09ECF8C8181111E
:105D50001CC00E94E20C98CF843009F095CF8C8152
:105D600020E0409187076D810CC04C8128E7429F5D
:105D7000040E40E0411D11248091850720E06091D0
:105D8000860790E00E941C0D7FCF0E94D50C60E03A
:105D90008C810E94EE0C78CF8C818093880780E004
:105DA0000E946D0A71CF8B81833031F170F48130A4
:105DB000B1F0823009F068CF80918407982F9370FA
:105DC000C9F0869586958C835FCF843009F05CCFCF
:105DD000809185078C83809186078D8355CF809134
:105DE00087072FEF829FC001112468E770E031D54B
:105DF0006C834ACF80E0E7CF80918807E4CF0E9490
:105E0000C61B42CF80E18A833FCF1A8287ED21CF24
:105E10004A805B80542445245424612C712C7E01DB
:105E20008FEFE81AF80A0C810E0D1F2D111DE016D8
:105E3000F10609F429CF87ED481651046104710475
:105E400078F4C201875D9C4F95D5F70184838FEF6D
:105E5000E81AF80A8FEF481A580A680A780AE7CF52
:105E600080E0F3CF9C80CA80DB80DC24CD24DC245E
:105E7000E12CF12C8E010F5F1F4F270132014914D5
:105E800051046104710408F0FFCE87EDC816D104F7
:105E9000E104F10430F4F8016481C601875D9C4F90
:105EA00085D58FEF481A580A680A780A8FEFC81A02
:105EB000D80AE80AF80A0F5F1F4FE1CF0E94521C70
:105EC000E3CE86E0A0CF9C80CA80DB80DC24CD249A
:105ED000DC24E12CF12C270132018E010B5F1F4FD6
:105EE000491451046104710408F0CECE80EDC81647
:105EF00082E0D806E104F10488F4C60189963AD517
:105F0000F80181938F018FEF481A580A680A780ABE
:105F10008FEFC81AD80AE80AF80AE2CF80E0F0CF7B
:105F20009C80CA80DB80DC24CD24DC24E12CF12C95
:105F30008E010F5F1F4F2701320149145104610484
:105F4000710408F0A1CE80EDC81682E0D806E10405
:105F5000F10428F4F8016481C601899627D58FEFF2
:105F6000481A580A680A780A8FEFC81AD80AE80A45
:105F7000F80A0F5F1F4FE1CF41E08C81811101C012
:105F800040E06B818A810E94AB1AB9CE2D813E819F
:105F900032272327322741E08C81811101C040E064
:105FA0006B818A810E94EA126FCE78941F921FB68D
:105FB0001F9211248F939F93AF93BF938091C70338
:105FC0009091C803A091C903B091CA030196A11D85
:105FD000B11D8093C7039093C803A093C903B093E6
:105FE000CA03BF91AF919F918F911F901FBE1F90C9
:105FF00018951F920F920FB60F9211242F933F9373
:106000004F935F936F937F938F939F93AF93BF93C0
:10601000EF93FF938091E10082FF09C08091E2003D
:1060200082FF05C08091E1008B7F8093E100809129
:10603000DA0080FF24C08091D80080FF20C08091CA
:10604000DA008E7F8093DA008091D90080FFA9C0AA
:1060500080E189BD82E189BD09B400FEFDCF81E008
:10606000809314078091B603811109C00E94FC102F
:106070000E94AD108091E20084608093E2008091E4
:10608000E10080FF1AC08091E20080FF16C080917D
:10609000E2008E7F8093E2008091E2008061809335
:1060A000E2008091D80080628093D80019BC85E01E
:1060B0008093140783E080938F018091E10084FF37
:1060C0002FC08091E20084FF2BC080E189BD82E176
:1060D00089BD09B400FEFDCF8091D8008F7D8093EB
:1060E000D8008091E1008F7E8093E1008091E200F2
:1060F0008F7E8093E2008091E20081608093E200D5
:106100008091B503811509F452C084E0809314078F
:1061100080911407843009F052C082E080938F018F
:106120008091E10083FF2CC08091E20083FF28C0B2
:106130008091E100877F8093E10082E080931407E3
:106140001092B5038091E1008E7F8093E1008091F1
:10615000E2008E7F8093E2008091E2008061809374
:10616000E20042E060E080E00E942D108091F000AB
:1061700088608093F00081E080938F0180938E018E
:10618000FF91EF91BF91AF919F918F917F916F910F
:106190005F914F913F912F910F900FBE0F901F90E5
:1061A000189519BC109214071092B60368CF80910D
:1061B000E30087FF02C083E0A9CF81E0A7CF81E0A1
:1061C000ADCF1F920F920FB60F9211241F932F93F2
:1061D0003F934F935F936F937F938F939F93AF936F
:1061E000BF93CF93DF93EF93FF93E9EEF0E08081CD
:1061F0001091EC008F7010FB112717F9182B1082EB
:10620000C0EFD0E08881877F888378940E940E1544
:10621000E9EEF0E010828881886088831F70108327
:10622000FF91EF91DF91CF91BF91AF919F918F91AE
:106230007F916F915F914F913F912F911F910F909F
:106240000FBE0F901F901895EF92FF921F93CF9360
:10625000DF93182FEB011092BC0084EA8093BC00FE
:106260000E94441D7C018091BC0087FF26C0809164
:10627000B900887F883029F08091B900887F80310B
:1062800089F51093BB0084E88093BC000E94441DF4
:106290007C018091BC0087FF1EC02091B900287F3F
:1062A00080E090E0283189F081E090E0203409F42A
:1062B00080E091958195910908C0C7010E94501D09
:1062C000C817D90780F68EEF9FEFDF91CF911F910E
:1062D000FF90EF900895C7010E94501DC817D9077D
:1062E000C0F6F1CF8FEF9FEFF0CF1092B9008CE0A6
:1062F0008093B80008950F931F93CF93DF93EB0122
:106300008093BB0084E88093BC000E94441D8C01F4
:106310008091BC0087FF10C02091B900287F81E0E8
:1063200090E0283209F480E0919581959109DF9100
:10633000CF911F910F910895CF3FDC0749F3C8011A
:106340000E94501DC817D90718F78EEF9FEFEFCFA7
:10635000A0E0B0E0EDEAF1E395C2982E862E772E0C
:106360006A0179010E94441D5C0184E1E816F10490
:1063700010F18FEFE816FE0409F1C70164E170E047
:1063800068D2162F072F612F702F892D5DDFEC014A
:10639000892BB1F4082D172DC00ED11E0C151D052B
:1063A00011F02097C1F084E98093BC00CE01CDB7F5
:1063B000DEB7EDE083C211E000E0E5CF15E0FCCFF1
:1063C0008FEFE816FE04F9F2C5010E94501DE81691
:1063D000F906C8F6DFCFB701F80181918F018BDF95
:1063E000EC01DCCFA0E0B0E0E7EFF1E34BC2982E88
:1063F000862E772E6A0189010E94441D5C010431BA
:10640000110500F10F3F100701F1C80164E170E0D0
:1064100020D2EB01BE01892D17DF7C01892BB9F455
:10642000C82DD72DCC0EDD1ECC15DD0519F0E114DD
:10643000F104B9F084E98093BC00C701CDB7DEB7A1
:10644000EDE03CC2C1E0D0E0E5CFC5E0FCCF0F3FBE
:10645000100701F3C5010E94501D08171907D0F657
:10646000DFCFFE018491B80146DF7C012196DCCFAD
:10647000A0E0B0E0EDE3F2E304C2982E862E742E85
:10648000652E6901E8010E94441D5C01043111057B
:1064900008F10F3F100711F1C80164E170E0D9D194
:1064A000F62EE72E6F2D7E2D892DCEDE8C01892BC9
:1064B000C1F0CF3FDC07B1F3C5010E94501DC817E2
:1064C000D90780F784E98093BC00C801CDB7DEB757
:1064D000EEE0F3C1FF24F394E12CE4CF85E0F82E45
:1064E000FBCFBE01882D07DF8C01E72CF62CCE0CEC
:1064F000DF1CEC14FD0431F30115110519F7BE0181
:10650000F70181917F01F7DE8C01F3CF8EE14A9B89
:1065100002C08150E1F74A9BFECF08955A9880E26D
:106520008A95F1F75A9A0895FC018BE08A95F1F764
:1065300028E080E090E031E040E14A95F1F7880FF3
:106540004A9B02C08160932742E04A95F1F7000020
:1065500040E14A95F1F7215079F720E12A95F1F7CA
:1065600029B132E03A95F1F7000030E13A95F1F7C0
:1065700031E022FD93272081920F90830895A1E0BE
:10658000B0E0E4ECF2E385C119828C017C01E60EF7
:10659000F11CBCDFCE010196C7DFF80181938F01AA
:1065A000EE15FF05B1F781E09981911180E0219608
:1065B000E6E08BC1529A5A9A089552985A9AEA9AEA
:1065C000E9E6F0E080818F7C808308956150770B4D
:1065D00091E001C0990F6A95EAF7692F90E021E0F8
:1065E000611108C0911591F05A9A80E28A95F1F7ED
:1065F0005A980895362F382339F05A9A922730E264
:106600003A95F1F76695ECCF5A98F9CF5A98EDCFB5
:10661000FF920F931F93CF93DF93EC018C01060F32
:10662000111D8991F82E7ADF68E08F2DCFDFC0171A
:10663000D107B9F7CDB7DEB7E5E048C11F920F9299
:106640000FB60F9211240F931F932F933F934F93E5
:106650005F936F937F938F939F93AF93BF93EF93CA
:10666000FF93CF93DF930F92CDB7DEB719824EDF42
:10667000CE01019659DF082F069506950695282F1D
:1066800022952570902F9570920F292F2370969543
:106690009695920F982797708981892B09F055C09C
:1066A0000E3008F052C080E18A95F1F75A9A529A5A
:1066B00082E08A95F1F700C05A9888E0089F80012F
:1066C0001124D801AC5DBE4F1696ED91FD9118973F
:1066D000309791F0609111037091120314962D91EF
:1066E0003D91260F371F15978D919D91680F791F4A
:1066F0004C9113978C910995F801EC5DFE4F6381E5
:10670000611549F020911103309112038481958124
:10671000820F931F7DDF02DF80E18A95F1F75A989F
:1067200052985A9A80E18A95F1F7F801EC5DFE4F94
:106730006081611549F0209111033091120381812C
:106740009281820F931F1BDFE1DE0F90DF91CF91CB
:10675000FF91EF91BF91AF919F918F917F916F9139
:106760005F914F913F912F911F910F910F900FBE0D
:106770000F901F9018950F931F93CF93DF93EC0109
:106780000E970CF05EC0F894529A5A9885E08A955C
:10679000F1F700009C2F969595708C2F8570980FBF
:1067A000892F837096959695292F93E0CC0FDD1F46
:1067B0009A95E1F7280F822F8C2B082FAFDE00C0AF
:1067C00068E0802F03DF80E18A95F1F752985A9AAA
:1067D0004A9B30C087E090E04A992EC0FE01EC5DF4
:1067E000FE4F6381611559F020911103309112031E
:1067F00084819581820F931FC2DE8115F9F086DEB8
:1068000080E28A95F1F75A98529A80E18A95F1F7D9
:10681000CC5DDE4F6881611549F020911103309104
:10682000120389819A81820F931FF2DE77DE7894BA
:1068300081E008C000C0CCCF019749F4529A5A9A1F
:10684000789480E0DF91CF911F910F91089500C05F
:10685000C3CFAA1BBB1B51E107C0AA1FBB1FA617B2
:10686000B70710F0A61BB70B881F991F5A95A9F7F9
:1068700080959095BC01CD0108952F923F924F9243
:106880005F926F927F928F929F92AF92BF92CF92C0
:10689000DF92EF92FF920F931F93CF93DF93CDB7C9
:1068A000DEB7CA1BDB0B0FB6F894DEBF0FBECDBF41
:1068B00009942A88398848885F846E847D848C8412
:1068C0009B84AA84B984C884DF80EE80FD800C811B
:1068D0001B81AA81B981CE0FD11D0FB6F894DEBFFE
:1068E0000FBECDBFED01089597FB072E16F400945F
:1068F00006D077FD08D0ADDF07FC05D03EF49095BB
:1069000081959F4F0895709561957F4F0895EE0F83
:10691000FF1F0590F491E02D0994692796276927B8
:106920007827872778270895FB01DC0104C08D9123
:106930000190801921F441505040C8F7881B990BF1
:106940000895FB01DC0102C001900D9241505040BE
:10695000D8F70895DC01CB01FC01F999FECF06C000
:10696000F2BDE1BDF89A319600B40D92415050400D
:10697000B8F70895F999FECF92BD81BDF89A99278D
:1069800080B50895A8E1B0E042E050E0E5CFDC0139
:10699000A40FB51F4150504040F0CB01840F951F0C
:1069A0002E9105D041505040D8F70895262FF999DF
:1069B000FECF92BD81BDF89A019700B4021639F05E
:1069C0001FBA20BD0FB6F894FA9AF99A0FBE08952F
:1069D0000396272FECDFEADF252FE9DF242FE7CF0F
:1069E0000196272FE4DFE2CFF894FFCF5D0B820BF7
:1069F000860B890B8C0B8F0B090C3E0CEC151216B9
:106A000018161216181666168816181682178F177B
:106A100012247A241A24E423E8231E24EC232224BB
:106A20002E24F8237324FC233224002436245B24F0
:106A300004243A2462240A2440244824F0232624EF
:106A4000F4232A240E24442452246B247124DE23AC
:106A500016248124BB23BF23B223B723C323C72318
:106A6000CB23C524CB249B249F24CE24A424D3242D
:106A7000A924D824AE24DD24B324E224E724EC2482
:106A80009B249F24CE24A424D324A924D824AE2438
:106A9000DD24B324E224272E2B2E682E7A2E852E79
:106AA000902E932E932E932E332E332E022F052FBE
:106AB000082F322F5E2F612F632F902FBC2FC62FF0
:106AC000E10039000021007F220003490003FFFF9D
:106AD00000FF00390501F4F5940F9012A312CF0FB7
:106AE000A81288120000000100000000000000054C
:106AF0000100000005060000000000000000000189
:106B00000B000000000000080C0000000000000066
:106B1000000031090414000000000000011800000A
:106B2000000000000119000000000000011A000030
:106B300000000000091B000000000000012400000C
:106B4000000000000C250000000000000000010013
:106B50006E147E14BC1400000001FF00FF78442274
:106B60006D3B011901AC009101AA01CA0100081096
:106B70001818100800FF0502000B0C15161F200A3C
:106B80000D14171E21090E13181D22080F12191CAF
:106B9000230710111A1BFF2F30393A43442E313886
:106BA0003B42452D32373C41462C33363D40472B46
:106BB00034353E3FFF60281014300A5012583C38DC
:106BC00039183C2039003000240018000C100C103B
:106BD000181024103030374039202D202120152066
:106BE0000930073013301F302B503B6040402D40A0
:106BF0002140154009500A50165022502F8028D0AD
:106C000014B00A9012883CA839C83CC039E030E082
:106C100024E018E00CD00CD018D024D030B037A02D
:106C200039C02DC021C015C009B007B013B01FB0C6
:106C30002B903B8040A02DA021A015A009900A9088
:106C4000169022902F080202020202020404040499
:106C500004040404040404040404040404040404F4
:106C600004040404040404040408020202020202EC
:106C700004040404040404040404040404040404D4
:106C8000040404040404040404040404040031316E
:106C9000295A1B750A42415345004C4F5745520033
:106CA00052414953450041444A5553540000D502CE
:106CB000010101DA02010202E002010003E6020121
:106CC0000300FF0100010000FFFF0000010001FFC1
:106CD0000046076697C63435F6F731333236E200A0
:106CE000E900EA00B500B600B700CD008301CC0092
:106CF0008A01920194012102230224022502260224
:106D000027022A02B300B4006F0070009F01CB017C
:106D10009F02A002E200E900EA00B500B600B70059
:106D2000CD008301CC008A0192019401210223024B
:106D300024022502260227022A02B300B4006F00B3
:0A6D400070009F01CB019F02A0022A
:00000001FF
